:10800000004000205120010061F2000061F20000F8
:1080100061F2000061F2000061F200000000000067
:1080200000000000000000000000000061F20000FD
:1080300061F200000000000061F20000FD85000018
:1080400061F2000061F2000061F2000061F20000E4
:1080500061F2000061F2000061F2000061F20000D4
:1080600061F2000061F2000061F2000061F20000C4
:1080700061F2000061F2000061F2000061F20000B4
:1080800061F2000061F2000061F2000061F20000A4
:1080900061F2000061F2000061F2000061F2000094
:1080A00061F2000061F2000061F2000061F2000084
:1080B00061F2000061F2000061F2000061F2000074
:1080C00061F2000061F2000061F2000061F2000064
:1080D00061F2000061F2000061F2000061F2000054
:1080E00061F2000061F2000061F2000061F2000044
:1080F00061F200000D88000061F2000061F20000F2
:1081000061F2000061F2000061F2000061F2000023
:1081100061F2000061F2000061F2000061F2000013
:1081200061F2000061F200001DED000061F200004C
:1081300061F2000061F2000061F2000061F20000F3
:1081400061F2000061F2000061F2000061F20000E3
:1081500061F2000061F2000061F2000061F20000D3
:1081600061F200007104010061F2000061F20000A0
:1081700061F2000061F2000061F2000061F20000B3
:1081800061F2000061F2000061F2000061F20000A3
:1081900061F2000061F2000061F2000019F10000DC
:1081A00061F2000061F2000061F2000061F2000083
:0C81B00061F2000061F2000061F20000CA
:10840000FFFFFFFFFFFFFFFFFFFFFFFF7EF9FFFF03
:1084100010B5054C237833B9044B13B10448AFF3BE
:1084200000800123237010BD00C6FF1F0000000064
:10843000AC2401000C4B43B10C480D4910B5AFF30F
:1084400000800C48036823B910BD0A48036833B99B
:108450007047094B002BF7D0BDE810401847064B7A
:10846000002BF5D0184700BF00000000AC2401002D
:1084700004C6FF1F6CC5FF1F0000000080F31188B9
:1084800070472F4B41F238015A5842F478525A50F3
:108490002C4A927902F00C020C2A4FD041F244028D
:1084A0002949995003F558339A78110748BF9A78AB
:1084B000264944BF42F008029A70214B41F244021F
:1084C000995041F204015A5842F4803242F0C002FD
:1084D0005A501A6842F440221A6003F5E833242205
:1084E0005A701B4A80211170A2221A70DA7802F0A9
:1084F0001F02DA7007221A710C225A719A799207B8
:10850000FCD59A79D006FCD40E4B19469A7902F024
:108510000C02082AFAD14C225A718B7903F00C0311
:10852000082BFAD1074B1A4699794906FCD5222126
:108530001970937903F00C030C2BFAD1704700BF2C
:1085400000700440004006400000330100001301A9
:1085500000500640264B5A7902F0E0025A711A790F
:1085600002F0F8021A71A3F500531A7802F08C0297
:1085700042F050021A705A7802F09C0242F0400217
:108580005A709A7802F0E6029A701A4A0023137021
:1085900083F31188184B012283F8182383F81923D9
:1085A000022283F8582383F8592383F81D2383F884
:1085B0001E2383F81F2383F8202383F8212303221B
:1085C00083F82D2383F82F2383F8312383F8332373
:1085D00083F83523042283F83923052283F83A23CC
:1085E000062283F85723072283F84923704700BFE8
:1085F00000F0074000E0074000E100E0314A136866
:108600000133F0B51360304A1368013313602F4B08
:108610001A683AB11A68013A1A601B6813B92C4BF0
:1086200001221A702B4B1A6812B11A68013A1A60AB
:10863000294B5A68294B92B21A60294A1868116866
:10864000884223DD19681068264C091AB1F5004FDD
:1086500025480ADA1E6817682168D0E90045F61B2C
:108660007143641845EBE1750BE0196817682668DB
:10867000D0E90045C91BC1F580317143641A65EB2F
:10868000E175C0E900451B681360F0BD186811680A
:108690008842F8DA11681868124C091AB1F5004FCF
:1086A000114806DA16681F682168F61BD0E90045F4
:1086B000E3E711681F682668C91BD0E90045C1F5CA
:1086C0008031CDE71CC6FF1F04D0FF1F10CDFF1F58
:1086D0000CCDFF1F14CDFF1F009003402CCDFF1FBA
:1086E00028CEFF1F68CDFF1F70CDFF1F41F23C0257
:1086F00005498B5843F000738B50044B044A5A6071
:1087000007221A60704700BF0070044010E000E0CC
:1087100040190100014B1868704700BF1CC6FF1FBD
:108720001449154B41F23402072888BF002010B5C8
:1087300053F82030114CB4FBF3F48B5843F48063AE
:108740008B500F4B4FF400725A602D209A6006F048
:108750009FFD0C4B0022DA709A709A71DA725A718E
:10876000C4F30422E4B21A705C70DA7842F02C028E
:10877000DA7010BD00700440EC22010020AA440011
:108780000090044000A00640094A13685168013374
:10879000202B08BF00238B4208D0116811440872B7
:1087A0001360044AD37843F08003D370704700BF4E
:1087B00020C6FF1F00A006400A4B996ADA6A914260
:1087C0000DD09A6A511C1A44996292F830200270B6
:1087D0009A6A202A01D100229A6201207047002063
:1087E000704700BF20C6FF1F044B1A7802F0FF003D
:1087F00012B100221A700120704700BF0CCDFF1F7C
:10880000014B1865704700BF20C6FF1F30B52648D2
:108810000179C9B28C0617D5244BDA6A9C6A0132F9
:10882000202A08BF0022A2421BBFDC6AC579C27998
:1088300018191EBFEDB280F83050DA621C4A0520CC
:1088400010601A6D1B4B1A604A0608D51A4B4FF47C
:1088500000329A60144AD37803F0BF03D3700B063A
:108860001BD5144B1868C0B9104B19685A6891424F
:1088700014D0114A4FF4003151605A68511C1A4407
:108880005960117A084AC9B2D1715968202908BFC4
:108890005860D37843F04003D37030BD024AD37898
:1088A00003F07F03F8E700BF00A0064020C6FF1FCB
:1088B00010CDFF1F14CDFF1F00F00F4062B67047B0
:1088C000FFF7FCBF72B67047FFF7FCBF4FF0E02325
:1088D00018B1034AC3F80C2D7047024AFAE700BFEB
:1088E0000400FA050100FA0510B9C90801F0E8BC56
:1088F0007047F7B5454A464E46494FF480731361B9
:1089000053619363D363136453647161B1604249EB
:1089100040F20310086048608860C8608862C862DE
:108920000B644B6401F5352140314FF44030486110
:1089300048603A493A480B6040F607044B608B6048
:10894000CB62446144603748374C036043608360C6
:10895000C460036100F53320C03014244461042452
:10896000446010248460314C636104F5322404F5C2
:1089700080742025656141F204042D4D2F5927F0A4
:10898000E0072F512F5947F0C0072F514FF4A06433
:10899000CC6013603446D360082600230A211A46AF
:1089A000B4461F46A646C4F804C00197019DB5F51C
:1089B0007A7F21D3DEF81050A660ED0748BF013260
:1089C0000197019DB5F57A7F1AD3DEF81050ED07B7
:1089D00058BF01330139E6D10A2A164A14D10A2BAD
:1089E00012D101231370094B4FF4E0621A60DA6070
:1089F0001023436003B0F0BD019D01350195D5E71B
:108A0000019D01350195DCE70023EBE70090044070
:108A100000F00F402880030000A0044000B0044094
:108A200080F00F4000C004400001090000D0044065
:108A30000070044064CDFF1FF7B5114B1B78E3B104
:108A400010491148114D20231E4600240F4686462A
:108A50004E6086600194019AAA420AD9BB60CEF8A2
:108A600004300194019AAA42F2D8019A013201928B
:108A7000F8E7019A01320192EDE703B0F0BD00BFC3
:108A800064CDFF1F00F00F4000F10F401FA1070051
:108A9000072809D8DFE800F004090C0F1114161894
:108AA0004FF400420A4B5A6070474FF48032F9E7A6
:108AB0000222084BF7E70822FBE74FF40062F8E7D1
:108AC0000122F6E70422F4E74FF48062F1E700BFE9
:108AD00000F00F4040F00F40072809D8DFE800F011
:108AE00004090C0F111416184FF400420A4B9A6037
:108AF00070474FF48032F9E70222084BF7E708226B
:108B0000FBE74FF40062F8E70122F6E70422F4E7FE
:108B10004FF48062F1E700BF00F00F4040F00F40DB
:108B200010B50021044644FA01F3DB07C8B205D5AD
:108B3000FFF7AEFF01310829F5D110BDFFF7CCFFDB
:108B4000F8E708B506282CD8DFE800F0040D121766
:108B50001C212600002006F025F9B0F5806F34BFF7
:108B60000020012008BD104B186900F0010008BD6D
:108B70000D4B1869C0F3800008BD0B4B1869C0F39A
:108B8000802008BD084B1869C0F3400008BD064BA3
:108B90001869C0F3C00008BD034B1869C0F3C020BA
:108BA00008BD002008BD00BF40F00F4007282DD8A9
:108BB000DFE800F004090E13181D2227144B186873
:108BC000C0F3C0307047124B1868C0F300407047C4
:108BD000104B1868C0F3400070470E4B1868C0F384
:108BE000C00070470B4B1868C0F3C0207047094B9A
:108BF000186800F001007047064B1868C0F3800049
:108C00007047044B1868C0F38020704700207047FD
:108C100000F00F4040F00F4070B5002425460126BB
:108C2000E0B2FFF78EFF18B106FA04F31D43EDB270
:108C30000134082CF4D1284670BD10F0010F314BDF
:108C400033D05A6942F002025A614FF400329A60FE
:108C500010F0020F2C4A30D0596941F008015961D7
:108C60000221916041072FD5596941F40061596192
:108C70004FF40061916001072ED5596941F001015F
:108C800059614FF480319960C1062DD5596941F081
:108C9000040159610121916081062CD5596941F483
:108CA000806159610423936070474FF400325A6029
:108CB0005A6922F002025A61CAE7022151605969D9
:108CC00021F008015961CDE74FF400615160596905
:108CD00021F400615961CEE74FF480315960596940
:108CE00021F001015961CFE701215160596921F05B
:108CF00004015961D0E7042151605A6922F480626D
:108D00005A61704740F00F4080F00F401B4B5A688B
:108D100010F0010F14BF42F0030222F001025A606A
:108D2000DA6881074CBF42F0030222F00102DA60E8
:108D3000124BDA6A10F0040F14BF42F0030222F063
:108D40000102DA621A6801074CBF42F0030222F006
:108D500001021A60094B9A6810F0100F14BF42F01C
:108D6000030222F001029A609A6A81064CBF42F027
:108D7000030222F001029A62704700BF00A0044083
:108D800048B9064BD3F8A020120705D50822C3F82E
:108D9000A020012070470020704700BF00C00440A1
:108DA00008B5082005F0FEFF5E2810D9124B1A788E
:108DB0000AB901221A70082005F0F4FF63280ED9C1
:108DC0000E4B1B785BB90E4B04229A6008BD08203D
:108DD00005F0E8FF5428EED80022074BEAE7082008
:108DE00005F0E0FF542802D9044B1B7813B1044B63
:108DF00004225A6008BD00BF74C6FF1F4CCDFF1F80
:108E0000C0F00F40034B1878013801288CBF0020B8
:108E10000120704774C6FF1F034B1878012806BF56
:108E200002221A700020704774C6FF1FC0B201F002
:108E300071BBC0B201F064BB08B508F03DF906F0A3
:108E4000FBFB06F0ABFBBDE8084008F0B7B938B54E
:108E5000054606F0F9FA08280AD900242819013431
:108E600006F072FB092CF9D106F0A2FB012038BDF7
:108E7000002038BD092106F007BB002006F094BD94
:108E80002149224841F23C028B5843F440538B5015
:108E90001F4B012119601A6802431A601D4ADA60EB
:108EA0001A61DA6A42F08052DA621A6822F001022C
:108EB0001A601A6822F000621A6003F5F8334FF462
:108EC00000721A615A619A61DA61A3F5F033196090
:108ED0001968014319601049D96001F52001196131
:108EE000D96A41F08051D962196821F001011960F5
:108EF000196821F00061196003F500331A605A60A7
:108F00009A60DA601A61704700700440000C1F809C
:108F100000C002400300013E0400513EFF281ED85D
:108F200000041E4B00F47C108AB141F0006108433C
:108F30005863DA6A002AFCDA184BDA6AD100FCD5E9
:108F4000986BDA6A42F01042C0B2DA62704741F0C0
:108F5000004108435863DA6A002AFCDAF0E7B0F50A
:108F6000007F18D200040E4B00F47C105AB141F07F
:108F7000006108435863DA6A002AFCDA084BDA6AAF
:108F8000D200FCD5DCE741F0004108435863DA6ABF
:108F9000002AFCDAD4E70020704700BF00C002407E
:108FA00000D00240C0EBC00038B500220C4600F5EE
:108FB000006503210120FFF7B1FF0022C5F307215F
:108FC0000120FFF7ABFF0022E9B20120FFF7A6FF67
:108FD000002211460120FFF7A1FF00221146207058
:108FE0000120FFF79BFF0022114660700120FFF770
:108FF00095FF00221146A0700120FFF78FFF00228D
:109000001146E0700120FFF789FF00221146207110
:109010000120FFF783FF0122607100211046FFF756
:109020007DFFA07138BD38B54FF4006401220621E0
:109030001046FFF773FF002205210120FFF76EFFA6
:10904000012200211046FFF769FF8007F3D50022B7
:1090500002210120FFF762FF0022C4F30721012053
:10906000FFF75CFF0022E1B20120FFF757FF002568
:10907000A5F13F014A424A41012000210135FFF795
:109080004DFF402DF4D1002205210120FFF746FFBE
:10909000012200211046FFF741FFC307F3D44034FB
:1090A000B4F5804FC2D138BDF7B5C0EBC00000F5B4
:1090B00000650C46002203210120FFF72FFFC5F3B6
:1090C000072100220120FFF729FFE9B20022012039
:1090D000FFF724FF002211460120FFF71FFF0022A7
:1090E000114607460120FFF719FF002211460646E8
:1090F0000120FFF713FF0022114605460120FFF76C
:109100000DFF002211468DF803000120FFF706FF36
:10911000002211468DF804000120FFF7FFFE012216
:109120008DF8050000211046FFF7F8FE23788DF832
:109130000600BB420ED16378B3420BD1A378AB4299
:1091400008D1DDF80300D4F80330C31A584258415F
:1091500003B0F0BD0020FBE7012238B504460D4600
:1091600010460621FFF7DAFE002205210120FFF755
:10917000D5FE012210460021FFF7D0FE8207F3D56D
:10918000002202210120FFF7C9FE0022C4F30721BB
:109190000120FFF7C3FE0022E1B20120FFF7BEFE6F
:1091A000012229461046FFF7B9FE002205210120C1
:1091B000FFF7B4FE012200211046FFF7AFFEC30700
:1091C000F3D438BD38B50D46C0EBC00404F50060DB
:1091D0000978FFF7C1FF697804F60100FFF7BCFFCB
:1091E000A97804F60200FFF7B7FFE97804F6030058
:1091F000FFF7B2FF297904F60400FFF7ADFF6979A4
:1092000004F60500FFF7A8FFA97904F60600BDE8FB
:109210003840FFF7A1BF2DE9F84316460122044666
:10922000884610460621FFF779FE0022052101201D
:10923000FFF774FE012200211046FFF76FFE85073D
:10924000F3D5002202210120FFF768FE0022C4F3BB
:1092500007210120FFF762FE0022E1B20120FFF7A3
:109260005DFE0025771EB5420DD1002205210120AB
:10927000FFF754FE012200211046FFF74FFEC307FF
:10928000F3D4BDE8F883013414F03F0918F8051051
:1092900039D0781B424242410120FFF73FFEB9F12D
:1092A000000F2ED1BD422CD2002205210120FFF754
:1092B00035FE012200211046FFF730FEC107F3D42E
:1092C000012206211046FFF729FE00220521012078
:1092D000FFF724FE012210460021FFF71FFE820740
:1092E000F3D5002202210120FFF718FE0022C4F36B
:1092F00007210120FFF712FE0022E1B20120FFF753
:109300000DFE0135AFE70122C6E710B50022044685
:1093100003210120FFF702FEC4F3072100220120F0
:10932000FFF7FCFDE1B200220120FFF7F7FD01226B
:1093300000211046BDE81040FFF7F0BDF8B5044627
:109340000E461546032100220120FFF7E7FDC4F376
:10935000072100220120FFF7E1FDE1B200220120F8
:10936000FFF7DCFD77193446013DBC4200D1F8BD62
:10937000A21BAB1A5A425A4100210120FFF7CEFD31
:1093800004F8010BF1E7F7B5002205210120FFF7F2
:10939000C5FD012200211046FFF7C0FD10F0710449
:1093A000F2D1FFF7B7F90546FFF7B4F9401B0028E3
:1093B000B8BF4042B0F5FA6F22DAC4B1334B1B7824
:1093C00003BB402232490020FFF7B8FF2022314979
:1093D0004020FFF7B3FF20222F496020FFF7AEFFA8
:1093E00020222E498020FFF7A9FF03B0F0BD40F2F4
:1093F000FF70FFF78AFFA0F1AA035C425C41D3E74C
:10940000002CDBD1002140F2FF70FFF7A5FEFFF733
:109410000AFE40221E49224F224E0020FFF7FBFE8B
:1094200040254FF480742046B4223946FFF7F3FEFE
:10943000B434284620223146FFF7EDFEB4F5477FCD
:1094400005F12005EFD102AD002345F8043D4FF4AE
:10945000C3642046042229460434FFF7DCFEB4F539
:10946000FF6FF6D1002301934FF4A7642046042236
:1094700029460434FFF7CFFEB4F5C36FF6D1AA2115
:1094800040F2FF70FFF768FE9BE700BF64CDFF1F4F
:109490000CC0FF1FC8CDFF1FE8CDFF1F08CEFF1F68
:1094A0003C2301001C2301002DE9F0411378C3F394
:1094B000411507460E46144615BB3D4A117BF9B9C6
:1094C000D8071DD45F2B1BD83A490978C1B913F0CE
:1094D000970F15D1DFF8E48098F800302BB1517A5E
:1094E0002846FFF701FA88F80050DFF8D48098F892
:1094F00000302BB1002001F00DF8002388F8003077
:109500000022217840F20110FFF708FD30700022A0
:10951000617840F20110FFF701FD70700022A17820
:1095200040F20110FFF7FAFCB070E178012240F23E
:109530000110FFF7F3FCF0702378D90735D45F2BC7
:1095400033D803F01E03082B11D0142B24D0062B84
:109550002BD124237B430C2707FB0537164DA2781C
:10956000E3783D4443EA02236B60BDE8F081A278D2
:10957000E378114943EA0223242257430C2202FBD9
:1095800005754B51A27812070FD56FEA03536FEAA6
:1095900013534B51BDE8F08124235F430C2303FB9D
:1095A0000575054BE2781D442A72BDE8F08100BFC5
:1095B000C8CDFF1F84CEFF1F78CDFF1F81CEFF1FB8
:1095C00087CEFF1F07B513788DF8013053788DF8DB
:1095D00000108DF8023001A993788DF803306A46A7
:1095E000FFF762FF03B05DF804FB07B58DF80010CC
:1095F0008DF801208DF802306A469DF810308DF804
:10960000033001A9FFF750FF03B05DF804FB07B575
:1096100000238DF800108DF801308DF8032013120F
:1096200001A96A468DF80230FFF73EFF03B05DF8EE
:1096300004FB5F292DE9F34180460F46144606D806
:1096400017F01E064FEA511113D0022E2ED023140C
:109650008DF801306A46231201A940468DF800704A
:109660008DF802308DF80340FFF71EFF02B0BDE811
:10967000F081032212FB0012244B2548120103EB58
:10968000020E9C50DEF80410651A002DB8BF6D4222
:10969000854208DD13448C424FF00102CCBF0C1808
:1096A0000C1A1A73D3E78EF80C60D0E7032616FB6A
:1096B0000016164D3601AA1955F806E05460AEEBB7
:1096C000040024F07F4300289360114BB8BF404250
:1096D000984217DD7445B4BF1B19E31A4A018DF88F
:1096E00000201A148DF801201A128DF8022001A909
:1096F0006A46404635448DF80330FFF7D5FE012316
:109700002B73A4E700231373A1E700BFBCCEFF1F98
:10971000FFFF7F0007B511F01C0204D1FFF789FF9E
:1097200003B05DF804FB00238DF800106A4601A920
:109730008DF801308DF802308DF80330FFF7B4FE5C
:10974000EEE70122114640F20110FFF7E7BB13B527
:10975000144602AA41F0010102F8041D6946FFF710
:10976000A3FE9DF8013023709DF8023063709DF8D0
:1097700000009DF80330A37002B010BD07B502AA27
:1097800041F0010102F8041D6946FFF78DFEBDF8A6
:10979000020040BA80B2030544BF6FEA00506FEA8E
:1097A000105003B05DF804FBF7B5490102AD4CB2AF
:1097B00044F0150305F8083D174601A92A46064658
:1097C000FFF772FE9DF805308DF8013044F0140467
:1097D0009DF806308DF800402A4601A930468DF8E4
:1097E00002308DF80370FFF75FFE03B0F0BDF7B5F0
:1097F000490102AD4CB244F0150305F8083D174687
:1098000001A92A460646FFF74FFE9DF805308DF860
:10981000013044F014049DF807308DF800402A46CA
:1098200001A930468DF802708DF80330FFF73CFE39
:1098300003B0F0BD73B502AC7F2304F8083D0D46BC
:10984000224601A90646FFF72FFE7E238DF8003041
:109850009DF805308DF8013005F00F059DF80730B3
:109860008DF80250224601A930468DF80330FFF7EB
:109870001BFE02B070BD2DE9F74F400145B2C1F3A8
:109880000A0845F0180101AA01F0F8010020FFF7CD
:109890005EFF9DF805404FEA141904F00F04A1453E
:1098A00040465CDC07F0E0FDA4EB0904064601201D
:1098B000A0400F4607F0E8FD0022334B07F04AFEB8
:1098C00002460B463046394607F06EFF08F07CF83A
:1098D00007F0ECFD2AA3D3E9002307F03BFE08F0D4
:1098E00073F807F0E3FD0022284B07F033FE4FF03A
:1098F000FF3906460F46CA4600244FF0010B0BFA0B
:1099000004F007F0C1FD3B46324607F023FE08F0A5
:1099100033F8A0F180037F2B98BFA14604F1010426
:1099200098BF82460E2CEAD1002445F0120101AA0C
:10993000204601F0F2018DF804408DF805A08DF865
:109940000690FFF73FFE45F00C012046424601F02D
:10995000EC01FFF75CFE204603B0BDE8F08F07F096
:1099600083FDA9EB040406460120A0400F4607F042
:109970008BFD02460B460020034907F015FF9FE7C9
:1099800004560E2DB29DEF3F0000604000002040C5
:1099900073B54A0803244FF4807314FB0233B424D4
:1099A00014FB0034064620460D46FFF7AEFC8DF84A
:1099B0000400601CFFF7A9FC8DF80500A01CFFF750
:1099C000A4FC45EA46118DF8060001AAC9B20020A0
:1099D000FFF7F8FD02B070BD73B50D4641EA4011C6
:1099E00001AA0646C9B20020FFF7B1FE03244FF4D6
:1099F00080736D0814FB0535B42414FB06549DF8E0
:109A000004102046FFF7A8FB9DF80510601CFFF727
:109A1000A3FB9DF80610A01CFFF79EFB02B070BDD3
:109A200010B5C4B221466401E4B202220020FFF75F
:109A3000BBFE44F008010020FFF76CFE44F00A0171
:109A40000020BDE81040FFF765BE37B5440144F083
:109A50001604E4B20D4601AA21460020FFF777FE66
:109A60009DF8053015F0010F14BF43F0400323F0BB
:109A700040038DF805309DF8053015F0020F14BF36
:109A800043F0100323F01003002001AA21468DF8B3
:109A900005308DF80600FFF795FD03B030BD37B5F2
:109AA000440144F01604E4B20D4601AA2146002008
:109AB000FFF74DFE9DF8053015F0010F14BF63F060
:109AC0007F0303F07F038DF805309DF8053015F016
:109AD000020F14BF43F0200323F02003002001AA4B
:109AE00021468DF805308DF80600FFF76BFD03B0B9
:109AF00030BD07B5410141F0160101AA01F0F601A0
:109B00000020FFF724FE9DF80530C3F38010DB062C
:109B100048BF40F0020003B05DF804FB07B5410107
:109B200041F0160101AA01F0F6010020FFF70FFE37
:109B30009DF80530D8099B0648BF40F0020003B0ED
:109B40005DF804FB70B5104C05016219204693685E
:109B50008B420DDACB1AC3F18076B342546804DC31
:109B6000234453602844816070BDA41B5460F9E70E
:109B7000F8DD5B1AC3F18076B342546801DCE31A66
:109B8000EFE73444F2E700BFBCCEFF1F73B502AA73
:109B900041F001030C4602F8043D69460546FFF713
:109BA00083FC9DF802009DF80110000240EA01408C
:109BB0009DF803100843030248BF40F07F405F2C2C
:109BC00005D8660914F01E0403D0022C08D002B098
:109BD00070BD032010FB05600001094B1858F6E723
:109BE00005EB4503334420F07F41D8B2FFF7AAFFCD
:109BF000032010FB0560024D05EB00156868E6E7E1
:109C0000BCCEFF1F38B50D4668210446FFF7BEFFE6
:109C10003DB140F0010220466821BDE83840FFF721
:109C200008BD20F00102F6E773B51C4B587E10F01A
:109C300001001DBF40F22312682100204FF49172F1
:109C400008BF6821FFF7F5FC0223009300231A46A2
:109C50007E211846FFF7C9FC00240025E6B2E9B2D0
:109C600030460135FFF794FE1D2DF8D17501EDB298
:109C700045F00C010020FFF789FF01463046FFF751
:109C8000FAFD013443F2FF1245F016010020FFF700
:109C9000BEFC032CE1D102B070BD00BF0CC0FF1FA1
:109CA0007FB5450104AA45F0030302F8043D0446CC
:109CB00002A90020FFF7F8FB9DF80A309DF8091073
:109CC0001B0243EA01439DF80B1020461943FFF79E
:109CD00039FF134A2301D118087BE8B111480C263B
:109CE00006FB0404267ABEB9D2584B680E48D41A33
:109CF000002CB8BF6442844210DD9A42CCBF1A18CF
:109D00001A1AD3B2009305F0E001C2F30723002032
:109D1000C2F30742FFF769FC04B070BD0E73F0E7B1
:109D2000BCCEFF1F78CDFF1FFFFF7F0038B5C0F30B
:109D30000741054600224FF48170FFF7EFF80C4C05
:109D4000000220600022C5F307214FF48170FFF765
:109D5000E5F823681843000220600122E9B24FF4BD
:109D60008170FFF7DBF8236818430009206038BDD5
:109D700078C6FF1F10B5244CC00023181A79032A97
:109D800084BF03221A7123189A79032A84BF0322FD
:109D90009A7123181A7A0F2A84BF0F221A72231875
:109DA0005A7A072A84BF07225A7223189A7A0F2AEE
:109DB00084BF0F229A72221813795279DB0343F47D
:109DC0000021E16012B143F40423E3602318DB793E
:109DD0001BB1E36843F40053E3602044037A8279C3
:109DE000DB0143EAC223E2681343427A43EA0213E7
:109DF000C27AE36012B9827A1343E360E068FFF746
:109E000095FFE368236110BD78C6FF1F10B5104CA5
:109E10000023C000E36023185B7E13B14FF400738E
:109E2000E36023189B7E1BB1E36843F48073E36017
:109E300023182044DA7E0F2A84BF0F22DA76C07EF0
:109E4000E3681843E060FFF771FFE368E36110BD6A
:109E500078C6FF1F38B5C2001F4C111A214491F873
:109E6000213091F8205091F822101B0343EA8533EA
:109E700043F46025012908BF2B46A2EB000108BF6F
:109E800043F480632144E56008BFE360E36891F830
:109E9000235091F8241043EA05230129E36004BF0D
:109EA00043F08003E360131A2344121A93F8253019
:109EB000012B08BFE368224404BF43F04003E36082
:109EC000E06892F8263040EA0310E060FFF72EFFCA
:109ED000E368A36238BD00BF78C6FF1F10B543001A
:109EE0001C4C1A18224492F92D103F29C4BF3F215F
:109EF00082F82D101A18224492F92D103F31BCBF60
:109F0000C12182F82D101A18224492F82E101F2910
:109F100084BF1F2182F82E104FF44022E2601A18ED
:109F20002244034492F82C202344012A04BF4FF416
:109F30005022E26093F82D00E26893F82E30000280
:109F4000134300F4FE401843E060FFF7EFFEE368C0
:109F5000236310BD78C6FF1F10B58300244C1A1868
:109F6000224492F83410012984BF012182F8341070
:109F70001A18224492F83510032984BF032182F86D
:109F800035101A18224492F836100F2984BF0F2179
:109F900082F836101A18224492F83710032984BF29
:109FA000032182F837101A182244034492F838101B
:109FB0000F29234484BF0F2182F8381093F838000A
:109FC00093F8342040F4202040EAC23093F8352042
:109FD00040EA423093F8362093F8373040EA0220C6
:109FE00040EA4310E060FFF7A1FEE368E36310BDC1
:109FF00078C6FF1F214B012010B503210024052244
:10A0000083F82C0083F825000220597283F8201071
:10A0100083F8211018729A72DC7283F82D2083F86D
:10A020002E2083F8224083F8234083F8244083F8CD
:10A03000260083F8344083F8354083F8364083F8AF
:10A04000374083F838405C769C76DC7618715C711A
:10A05000DC719C710A4B04229A602046FFF77CFF5A
:10A060002046FFF73BFF2046FFF7F4FE2046FFF7B0
:10A07000CDFE2046BDE810407CE600BF78C6FF1F3D
:10A08000C0F00F40044B042903EBC00318BF0022AB
:10A09000D97618BF5A76B9E678C6FF1F034B03EB93
:10A0A000C003597609B10422DA76AFE678C6FF1FFD
:10A0B000024B03EBC0039976A8E600BF78C6FF1FEA
:10A0C000024B03EBC000C07E704700BF78C6FF1F85
:10A0D000024B03EBC000407E704700BF78C6FF1FF5
:10A0E000024B03EBC000807E704700BF78C6FF1FA5
:10A0F000024B03EBC00319713CE600BF78C6FF1F9B
:10A10000024B03EBC003597134E600BF78C6FF1F52
:10A11000024B03EBC003D9712CE600BF78C6FF1FCA
:10A12000024B03EBC003997124E600BF78C6FF1F02
:10A13000024B03EBC00319721CE600BF78C6FF1F79
:10A14000024B03EBC003597214E600BF78C6FF1F31
:10A15000024B03EBC00399720CE600BF78C6FF1FE9
:10A16000024B03EBC0000079704700BF78C6FF1FA9
:10A17000024B03EBC0004079704700BF78C6FF1F59
:10A18000024B03EBC000C079704700BF78C6FF1FC9
:10A19000024B03EBC0008079704700BF78C6FF1FF9
:10A1A000024B03EBC000007A704700BF78C6FF1F68
:10A1B000024B03EBC000407A704700BF78C6FF1F18
:10A1C000024B03EBC000807A704700BF78C6FF1FC8
:10A1D000034B00EB8002134483F83410BCE600BF4D
:10A1E00078C6FF1F034B00EB8002134483F8351041
:10A1F000B2E600BF78C6FF1F034B00EB800213449A
:10A2000083F83610A8E600BF78C6FF1F034B00EBAB
:10A210008002134483F837109EE600BF78C6FF1F04
:10A22000034B00EB8002134483F8381094E600BF20
:10A2300078C6FF1F034B00EB8000184490F83400F1
:10A24000704700BF78C6FF1F034B00EB8000184427
:10A2500090F83500704700BF78C6FF1F034B00EB36
:10A260008000184490F83600704700BF78C6FF1F82
:10A27000034B00EB8000184490F83700704700BF94
:10A2800078C6FF1F034B00EB8000184490F838009D
:10A29000704700BF78C6FF1F034B00EB400213441A
:10A2A00083F82C101AE600BF78C6FF1F034B00EBA3
:10A2B0004002134483F82D1010E600BF78C6FF1F3C
:10A2C000034B00EB4002134483F82E1006E600BF58
:10A2D00078C6FF1F034B00EB4000184490F82C0099
:10A2E000704700BF78C6FF1F034B00EB40001844C7
:10A2F00090F92D00704700BF78C6FF1F034B00EB9D
:10A300004000184490F82E00704700BF78C6FF1F29
:10A31000034BC0EBC002134483F820109AE500BF42
:10A3200078C6FF1F034BC0EBC002134483F8211013
:10A3300090E500BF78C6FF1F034BC0EBC00213447B
:10A3400083F8221086E500BF78C6FF1F034BC0EBE1
:10A35000C002134483F823107CE500BF78C6FF1FBA
:10A36000034BC0EBC002134483F8241072E500BF16
:10A3700078C6FF1F034BC0EBC002134483F82510BF
:10A3800068E500BF78C6FF1F034BC0EBC002134453
:10A3900083F826105EE500BF78C6FF1F034BC0EBB5
:10A3A000C000184490F82000704700BF78C6FF1F17
:10A3B000034BC0EBC000184490F82100704700BF69
:10A3C00078C6FF1F034BC0EBC000184490F8220072
:10A3D000704700BF78C6FF1F034BC0EBC000184496
:10A3E00090F82300704700BF78C6FF1F034BC0EBF7
:10A3F000C000184490F82400704700BF78C6FF1FC3
:10A40000034BC0EBC000184490F82500704700BF14
:10A4100078C6FF1F034BC0EBC000184490F826001D
:10A42000704700BF78C6FF1F2DE9F0479046334ABA
:10A43000089F099E1D461318044693F8403089462C
:10A440009246042B2FD8DFE803F0031A20262C00B5
:10A45000FFF790FC0AEB04030122C4EBC40454444C
:10A4600083F8402094F82630012B31D01FD3022BE3
:10A4700035D016B1DAF800303370BDE8F087FFF759
:10A48000E9FC0AEB04030222E7E7FFF765FD0AEBAC
:10A4900004030322E1E7FFF721FD0AEB0403042292
:10A4A000DBE7FFF7B3FC0AEB04030022D5E7B9F1C1
:10A4B000000F04D0DAF800309B0C89F80030B8F1B6
:10A4C000000FD6D0DAF800309B0A88F80030D0E7C9
:10A4D000002DCED0DAF800309B0A2B60C9E725B1F9
:10A4E000DAF80030DB0B5B012B60002FC1D0DAF80B
:10A4F0000030C3F384233B70BBE700BF78C6FF1F67
:10A5000028B9034BDA7A12B90122DA7232E47047C1
:10A5100078C6FF1F20B9034BD97A09B1D87229E454
:10A52000704700BF78C6FF1F062808D8DFE800F094
:10A5300004080B0E111417000A4B1B680B607047C0
:10A54000084BDB69FAE7074B1B69F7E7054BDB6B49
:10A55000F4E7044B1B6BF1E7024B9B6AEEE7014B00
:10A56000DB7AEBE778C6FF1F13B5C74C63789A1FF9
:10A57000012A11D98C2B0FD0C02B0DD0C72B0BD09B
:10A5800003F16002D2B2182A06D903F13402D2B222
:10A59000322A07D8D52B05D0A27832B10422BB4B82
:10A5A0001A7047E1A278022AF8D8A42B00F065823D
:10A5B00000F2A680842B00F0488148D8062B00F0DA
:10A5C0007B8119D8022B00F0408107D8002B00F0C6
:10A5D0002881012B00F030810322E0E7042B23D0F7
:10A5E00040F25E81D4F80310A078FFF744F9A37815
:10A5F000D4F80310A64A26E0802B00F012810ED872
:10A600000C2B00F060810D2B00F07E81072BE3D135
:10A61000A278A04B03EB4213E2789A720AE1822BF4
:10A6200000F0878140F20881A178D4F80320490125
:10A6300041F0060101F0E6010020FEF7E8FFA378F3
:10A64000D4F80310944A42F82310002118E1942B07
:10A6500000F0398128D88A2B00F074810ED8862B1F
:10A66000C0D0C0F01D81872BB6D1A178D4F80320CB
:10A67000490141F00E0101F0EE0119E18D2B00F0CE
:10A680006F81932B00F040818C2BA5D1E178A078CD
:10A69000C1F10801C9B2FFF7F5FCA2787D4B03EBCD
:10A6A0004213E278DA72C5E0A02B00F0D1811BD80A
:10A6B000992B00F061819A2B00F07A81952B8BD138
:10A6C000A178490141F0140101AA01F0F401002030
:10A6D000FFF73DF8D4F803209DF80530002A00F07C
:10A6E000488143F00403FFE0A22B00F0BF8140F259
:10A6F000B681D4F80310A078C9B2FFF701FD99E044
:10A70000B52B00F015823ED8AC2B00F0E0811BD8B1
:10A71000A82B00F0C7810BD8A62B00F0BC8140F21B
:10A72000B381D4F80310A078C9B2FFF711FD81E01E
:10A73000AA2B00F0C58140F2BC81D4F80310A078A8
:10A74000C9B2FFF763FD75E0B02B00F0DC810BD8D8
:10A75000AE2B00F0D18140F2C881D4F80310A0786C
:10A76000C9B2FFF7D5FD65E0B22B00F0DA81C0F089
:10A77000D181B32B7FF430AFD4F80310A078C9B2E5
:10A78000FFF7F8FD56E0C72B00F0968022D8C02BCB
:10A790003FF43EAF0ED8B72B00F0E381C0F0D2817A
:10A7A000B82B7FF419AFD4F80310A078C9B2FFF723
:10A7B000AFFC3FE0C22B00F01481C0F00B81C32B33
:10A7C0007FF40AAFA278334B03EB4213D4F8032093
:10A7D0005A602FE0D42B00F0248110D8D12B00F048
:10A7E0000781D22B00F00A81CC2B7FF4F5AEA27842
:10A7F000284B03EB4213D4F80320DA811AE0D62B5E
:10A8000000F01E81C0F01581FE2B7FF4E5AE214BD8
:10A81000A178D4F8032003EB411302B101221A738B
:10A8200008E0A178D4F80320490101F0E0010020FC
:10A83000FEF7FFFE02B010BDA178D4F80320490155
:10A8400041F0020101F0E201F1E7A178D4F8032020
:10A85000490141F0080101F0E8010020FEF7D7FEB0
:10A86000A178D4F803204901002A41F0060101F043
:10A87000E601B8BF52420020FEF7C9FEA3780121CD
:10A88000064AD154D6E700BFECCEFF1F08D0FF1F09
:10A8900014D0FF1FC8CDFF1F20D4FF1FBCC6FF1F51
:10A8A000A178D4F80320490141F00A0101F0EA013E
:10A8B0000020FEF7ACFEBDE7A278AE4B03EB4213DF
:10A8C000E2785A72B6E7A178490141F0140101AA71
:10A8D00001F0F4010020FEF73AFFD4F803209DF8C0
:10A8E000053072B143F002038DF80530A1784901BB
:10A8F00041F0140101AA01F0F4010020FEF762FE0C
:10A9000098E723F00203EFE7A178490141F0140131
:10A9100001AA01F0F4010020FEF719FFD4F803208A
:10A920009DF8053012B143F00103DDE723F0010388
:10A93000DAE7A178D4F80320490141F0040101F0DD
:10A94000E401B5E7A178490141F0140101AA01F041
:10A95000F4010020FEF7FBFEE3788DF80630C5E732
:10A96000A178D4F80320490141F01A0101F0FA015D
:10A970009EE723F00403B7E7A178490141F01801ED
:10A9800001AA01F0F8010020FEF7E1FE9DF8053074
:10A99000E27823F00F0302F00F021343A1788DF841
:10A9A0000530490141F0180101AA01F0F801A4E7BE
:10A9B000A178490141F0180101AA01F0F801002035
:10A9C000FEF7C5FE9DF80530E27803F00F0343EA79
:10A9D0000213E3E7A278674B03EB4213E2781A72A3
:10A9E00028E7A378634AD4F803105B01D15021E72C
:10A9F000D4F80310A07804F0CFFB1BE7A0785D4BE0
:10AA0000E178D4F8032003EB401301F01F011A6131
:10AA100004F0B2FBD4F80310A078491104F0A4FBB1
:10AA200008E7A278534B03EB4213D4F803205A6192
:10AA300000E7A2784F4B03EB4213E2789A77F9E6EE
:10AA4000A2784C4B03EB4213D4F803209A83F1E62F
:10AA5000D4F80310A078C9B2FFF720FBEAE6D4F8D7
:10AA60000310A078C9B2FFF723FBE3E6D4F8031084
:10AA7000A078C9B2FFF73CFBDCE6D4F80310A0785D
:10AA8000C9B2FFF74DFBD5E6D4F80310A078C9B2E0
:10AA9000FFF74EFBCEE6D4F80310A078C9B2FFF75B
:10AAA0004FFBC7E6D4F80310A078C9B2FFF790FBBC
:10AAB000C0E6D4F80310A078C9B2FFF793FBB9E65B
:10AAC000D4F80310A078C9B2FFF796FBB2E6D4F829
:10AAD0000310A078C9B2FFF7A3FBA278264B03EBC3
:10AAE000C203D4F803205A71A4E6D4F80310A07866
:10AAF000C9B2FFF7D1FB9DE6D4F80310A07849B2A4
:10AB0000FFF7D4FB96E6D4F80310A078C9B2FFF79C
:10AB100009FC8FE6D4F80310A078C9B2FFF70CFC4B
:10AB200088E6D4F80310A078C9B2FFF70FFC81E6DD
:10AB3000A078104BD4F8032003EB40139A61FEF782
:10AB40001FF977E6A078D4F803200B4B43F83020A8
:10AB5000002A7FF46FAE03EBC0035979FFF760FB67
:10AB600068E6A278044B03EBC203D4F803201A7101
:10AB700060E600BFC8CDFF1F34CDFF1F37B5C04D05
:10AB8000C04C6B789A1F012A11D98C2B0FD0C02B87
:10AB90000DD0C72B0BD003F16002D2B2182A06D910
:10ABA00003F13402D2B2322A07D8D52B05D0AA78C5
:10ABB00032B10423237003B030BDAA78022AF8D83A
:10ABC000A32B00F03F8200F2BE80832B00F08B812C
:10ABD0005BD8082B00F0A58021D8032B00F07C81E6
:10ABE0000ED8012B00F0718140F26681A9784901ED
:10ABF00041F0080101F0E8010020FEF7BFFD62E12D
:10AC0000052B4ED0C0F06F81062B00F0FD80072B86
:10AC100039D1AA789C4B03EB42139B7AF9E00C2BB9
:10AC200000F0668114D80A2B00F0788140F26F8121
:10AC300001AA7C210020FEF78AFDAB785A0002238E
:10AC400093409DF80620134214BF01230023E0E047
:10AC5000802B00F0318110D80D2B14D1A978490137
:10AC600041F0140101AA01F0F4010020FEF76FFD8C
:10AC70009DF8053003F00103CBE0812B00F0258126
:10AC8000822B00F0568103236AE1942B00F030817F
:10AC900022D8872B00F0548106D8852B00F01C8128
:10ACA000A4D9AA78794B20E18C2B00F050810ED8E2
:10ACB0008A2BE8D1A978490141F0140101AA01F0D9
:10ACC000F4010020FEF743FD9DF80630A1E08D2B36
:10ACD00000F04881932BC0E79C2B00F01F811AD80D
:10ACE000992B00F0468110D8952BCCD1A978490139
:10ACF00041F0140101AA01F0F4010020FEF727FD44
:10AD00009DF80530C3F3800383E09A2B00F0408167
:10AD10009B2B8DD0B7E7A02B00F08C810AD89D2B00
:10AD2000B1D10020FEF70DFDAB785B00184100F0BB
:10AD30000100C8E0A12B00F08181A22BA3D1A8784B
:10AD4000FFF70EFABFE0B62B00F0B98142D8AC2B6A
:10AD500000F094811AD8A72B00F0808108D8A52B89
:10AD600000F0788140F27281A878FFF721FAAAE01A
:10AD7000A92B00F07B81C0F07581AA2B00F07A81AD
:10AD8000AB2B80D1A878FFF773FA9CE0B12B00F0D1
:10AD900087810ED8AE2B00F07B81C0F07581AF2B80
:10ADA00000F07A81B02B7FF46EAFA878FFF700FB3C
:10ADB00089E0B32B00F07C81C0F07681B42B00F0E9
:10ADC0007B81B52B7FF45FAFAA782F4B03EB421347
:10ADD0009B691EE0CC2B00F0FD802CD8C12B00F02D
:10ADE000E58006D8B82B00F07581C0F06D81C02BCE
:10ADF0000EE7C32B00F0E580C0F0DE80C42B00F02E
:10AE0000E680C72B7FF43FAFAA781F4B03EB4213BA
:10AE10005B7A63601E4B1B78002B3FF4CCAE1D4B5E
:10AE200062681A601C4B002A40F058811A6842F090
:10AE300008021A60BFE6D22B00F0EA8013D8CF2BAD
:10AE400000F0CE8005D8CE2B7FF41DAFAA78134B2F
:10AE50004BE0D02B00F0D880D12B7FF414AFA87832
:10AE600004F08EF92FE0D52B00F0D88018D8D42B21
:10AE70007FF409AFAA78044B03EB42135B69C8E780
:10AE8000ECCEFF1F08D0FF1FC8CDFF1F14D0FF1F3F
:10AE900003D0FF1FF4CFFF1FF4CEFF1F58CDFF1FBD
:10AEA000D62B00F0C180FE2B7FF4EDAEAA788D4B3F
:10AEB00003EB42131B7BACE7A978490101F0E001E9
:10AEC0000020FEF763FE6060A4E7A978490141F025
:10AED000020101F0E201F3E7A978490141F00A011A
:10AEE00001F0EA0188E6AA787F4B53F8223090E718
:10AEF000A978490141F0140101AA01F0F4010020F0
:10AF0000FEF725FC9DF80530C3F3400381E70020E0
:10AF1000FDF717FE003018BF0120D4E701AA7C21FD
:10AF20000020FEF714FCAA789DF806305200134169
:10AF3000A0E6A978490141F0040101F0E4015BE6D3
:10AF4000A978490141F00E0101F0EE0154E6AB7819
:10AF50002BB90020FFF7B4F8C0F10800B3E70423D1
:10AF6000237057E7A978490141F01A0101F0FA016D
:10AF700042E6A978490141F0180101AA01F0F8015F
:10AF80000020FEF7E4FB9DF8053003F00F0340E7D7
:10AF9000A978490141F0180101AA01F0F801002047
:10AFA000FEF7D5FB9DF805301B0932E7AA784D4B1B
:10AFB00003EB42131B7A2CE7AB784A4A5B01D35868
:10AFC00027E7AA78474B03EB42135B6821E7AA788F
:10AFD000464B8AE7AA78434B03EB4213DB8918E719
:10AFE00000236360424AAB78D15C09B10121616002
:10AFF0000021D1543F4AD15C19B1616841F002018E
:10B0000061600021D15405E7AB783B4AD35C00E78F
:10B01000AA78344B03EB42131B69FAE6AA78314B4A
:10B0200003EB42139B7FF4E6AA782E4B03EB42130B
:10B030009B8BEEE6A878FFF74BF844E7A878FFF77C
:10B040004FF840E7A878FFF793F83CE7A878FFF7B8
:10B050009FF838E7A878FFF7A3F834E7A878FFF758
:10B06000AFF830E7A878FFF7E5F82CE7A878FFF706
:10B07000EBF828E7A878FFF7F1F824E7AA781F4B48
:10B0800003EBC2035B79C4E6A878FFF723F91AE75C
:10B09000A878FFF729F916E7A878FFF77FF912E7F4
:10B0A000A878FFF78FF90EE7A878FFF795F90AE778
:10B0B000A878FFF7A5F906E7AB78114AA6E7AA78C2
:10B0C0000E4B53F83230A4E6AA780C4B03EBC203C4
:10B0D0001B799EE6A878FFF753F8F4E61A6822F089
:10B0E0000802A6E6C8CDFF1F20D4FF1F1CCDFF1FFE
:10B0F000C0CDFF1F50CDFF1FC3CDFF1F34CDFF1F9D
:10B1000030CDFF1F38B5984A9378022B144600F0D3
:10B110002481032B00F03681002B40F00982537804
:10B120004E2B00F0C18031D8462B00F08F8012D812
:10B13000422B7BD006D8402B6CD0412B71D0032200
:10B140008A4B65E0442B76D0452BF8D1884BD178DB
:10B150005971052061E04B2B00F096800CD8472BED
:10B160007CD0492BEBD1D278814B002A40F08780EC
:10B17000DA75D97D172050E04C2B00F090804D2BD4
:10B18000DDD17B4BD1785975152046E0542B00F06A
:10B19000BD801BD8512B00F0A48009D84F2B00F0A4
:10B1A0008E80502BCBD1724BD1789975162034E01C
:10B1B000522B00F0A380532BC1D16D4DD2F8033038
:10B1C0002946042241F8103F10204FE0832B00F065
:10B1D000B58014D8552B00F0A580562BAFD1D2F8EE
:10B1E00003300F2B00F2A481D1780020FEF722FB60
:10B1F0005F49E37801F8243F0122242022E0852BD7
:10B2000000F0A680C0F09F80FF2B98D1D278594BD8
:10B210001A7038BDD17840F2FF70BDE83840FDF7B4
:10B220009BBF534BD17819700020F6E7504BD17873
:10B2300059700120F1E74E49D2F8033041F81C3F24
:10B2400004221C20BDE83840FDF7E5BF4849D2F88C
:10B25000033041F80C3F04220C20F3E7444DD2F8B0
:10B2600003302946042241F8083F0820FDF7D3FFA8
:10B270002A8A29896879BDE8384003F0C5BD3B4971
:10B280000122DA754A6074E7394CD178E170032005
:10B29000FDF762FFE078BDE83840FDF7B1BA344B06
:10B2A000D17899700220B8E7314CD2F80300E084DD
:10B2B000FDF7C3FC022204F126012620C2E7D2F8E2
:10B2C00003102B4CC9B219206176FDF745FF617E52
:10B2D00011F0010118BF01210020BDE83840FEF740
:10B2E00091BC234D2A7DD20704D5E378DB0701D436
:10B2F000FDF799FEE178297514208EE71C49D2F8F4
:10B30000033041F8203F042220209BE7D2F803308D
:10B31000012B00F20D811649D37801F81A3F012262
:10B320001A208FE7D2F80330012B00F20181104977
:10B33000D37801F81B3F01221B2083E70E4BD2F884
:10B3400003205A6038BD0D4BD2F803201A6038BD77
:10B35000094BD2F803209A6038BD5178084BD2F8D7
:10B36000032043F8212038BDECCEFF1F08D0FF1F7B
:10B370000CC0FF1F02D0FF1FBCC6FF1F04D0FF1F61
:10B3800020D0FF1F53782E2B3FF6D9AE01A252F8E2
:10B3900023F000BF51B4000063B4000075B4000096
:10B3A0003FB100003FB100003FB100003FB10000DD
:10B3B0003FB100003FB1000087B4000091B400002D
:10B3C0009BB400003FB100003FB100003FB100005E
:10B3D0003FB100003FB100003FB100003FB10000AD
:10B3E0003FB100003FB100003FB100003FB100009D
:10B3F0003FB100003FB100003FB100003FB100008D
:10B40000A5B40000B3B40000C1B40000C9B400008A
:10B41000D1B40000D9B400003FB100003FB100003A
:10B420003FB100003FB100003FB100003FB100005C
:10B43000E1B40000EBB40000F5B40000FFB400007C
:10B4400009B5000013B500001DB5000027B50000C8
:10B45000384BD4F803201A60FDF75CF9364BD860FE
:10B4600038BD344BD4F803205A60FDF753F9324B02
:10B47000186138BD2F4BD4F803209A60FDF74AF9C4
:10B480002D4B586138BD2B4BD4F80320DA6038BD02
:10B49000284BD4F803201A6138BD264BD4F803207A
:10B4A0005A6138BDD4F803100020BDE83840FEF7DB
:10B4B000CCBAD4F803100020BDE83840FEF7EFBA4C
:10B4C000D4F803100120F0E7D4F803100120F3E7CB
:10B4D000D4F803100220E8E7D4F803100220EBE7C9
:10B4E000144BD4F803209A6138BD124BD4F80320D2
:10B4F000DA6138BD0F4BD4F803201A6238BD0D4B0A
:10B50000D4F803205A6238BD0A4BD4F803209A625B
:10B5100038BD084BD4F80320DA6238BD054BD4F8A7
:10B5200003201A6338BD034BD4F803205A6338BD97
:10B53000042205E638CEFF1FBCC6FF1F2DE9F047E9
:10B54000804616460F4600294BD0002849D081423C
:10B5500047D0540164B244F00605EDB229460020FC
:10B56000FEF714FB44F00C0101F0EC0182460020D0
:10B57000FEF70CFB8146404606F02CFB044638469D
:10B5800006F028FB0146204606F030FC07465046F0
:10B5900006F020FB394606F029FC06F039FD04468A
:10B5A000484606F017FB394606F020FC06F030FD51
:10B5B000002C08BF01240C49002814BF80464FF01E
:10B5C0000108384606F0FCFC18B141463046FEF74B
:10B5D00052F9224629460020FEF72BF8034B0122A0
:10B5E0009A55BDE8F08700BF0000A041BCC6FF1F10
:10B5F00070B50C4D2B5C04469BB1C6B20A4B710171
:10B6000041F0060153F8202001F0E6010020FDF78B
:10B61000FEFF064B304653F82410FEF72CF90023AA
:10B620002B5570BDBCC6FF1F20D4FF1F14D0FF1FB9
:10B630002DE9F04FC44EC54F32787A7064233B70C9
:10B64000212AD6F803307B6085B034463D4601F0B0
:10B65000728300F2C1800E2A01F03D8039D8072A9A
:10B6600000F01C8414D8032A00F01C8208D8012A98
:10B6700000F09981022A00F0D68102232B70CFE1DD
:10B68000052A00F0088440F23E82FFF777FAC7E10E
:10B690000A2A00F0618607D8082A00F00885092ADE
:10B6A000EBD1FFF72FFDBBE10C2A00F0E18740F260
:10B6B000B087B078022800F202847378012B00F082
:10B6C000EF87C0F0E987022B00F0EE8703233B7081
:10B6D000A6E1182A01F041812BD8142A01F08A80B2
:10B6E00015D80F2A01F02080132AC6D17178984A04
:10B6F000092901F25380DFE811F04E085A085D086D
:10B70000600864086B086E08710874086908162AD6
:10B7100001F01F8141F28F808E4A116A072900F2E1
:10B720007F81481C02EB81011062D0694862D361BD
:10B7300076E11C2A01F00B8220D81A2A01F02B8115
:10B7400041F21881834D95F8452062B95E1C04BF13
:10B750007F4B1B680A205843A864FCF7DBFF0123DA
:10B76000E86485F845306378042B00F25981DFE8FE
:10B7700013F023095F098C09BD0937091F2A01F05D
:10B780001A8201F276821E2A7FF477AF7278142A29
:10B7900000F24F87B078022801F2DE8102EB42040A
:10B7A0006D4D044445F824306C4B9B7E002B00F01B
:10B7B0003781002A00F03481032111FB02010C23A0
:10B7C000013A5A4302F5C363042205EB810102FBEF
:10B7D0000030FDF720FD23E1802A01F0938344D857
:10B7E000402A01F0698329D8242A01F002830CD869
:10B7F000222A01F0F682232A7FF43FAF544B1B68C4
:10B80000C6F80330FFF77EFC0AE1262A01F02E83FA
:10B81000C1F02283272A7FF430AFB278022A00F2E7
:10B820004E837378142B00F2048703EB4303134415
:10B83000474A1168484A42F82310F1E0442A01F0CF
:10B84000558307D8422A01F03F8341F2398302F041
:10B85000D6F9E5E0462A01F05183C1F04B83472A2F
:10B860007FF40BAF02F0CFF9DAE0872A01F0DF8333
:10B8700046D8832A01F0628309D8812A01F04783E0
:10B88000822A7FF4FAAE334B02221A76C8E0852A68
:10B8900001F08683314A41F270833149314C0125F0
:10B8A0000D709178217040F2FE718B4201F27D8320
:10B8B000127D12EA050641F07883184601A9FDF7CA
:10B8C00071FB9DF8043063709DF80530A3709DF8FE
:10B8D0000630E3709DF80A3023719DF809306371DA
:10B8E0009DF80830A3719DF80730E37126722B464E
:10B8F000E15C227A01330A44082B2272F8D18FE0EE
:10B900008C2A01F0DA833BD8892A01F0BB83C1F08D
:10B9100056838A2A7FF4B1AE7278134B002A41F025
:10B92000C9831A70114AE37813700A4A92F83411E5
:10B930000F4A11700F4900220A700F490A700F4A0E
:10B9400011780B4313706BE0ECCEFF1F08D0FF1F84
:10B95000F4CFFF1FBCC6FF1FF8CEFF1F0CC0FF1F98
:10B96000F8CFFF1FF9CFFF1F28CDFF1F54CDFF1FBA
:10B9700080CEFF1F53CDFF1FB9CEFF1F29CDFF1F64
:10B98000F22A01F02184FF2A01F063848D2A7FF4DA
:10B9900074AE7278032A01F2FC83DFE812F0CF0B59
:10B9A000B60BE80BF60BB378022B00F28882DFF8B7
:10B9B000CC82DFF8C092DFF8B8A20026A278F5B2F8
:10B9C000AA4209D0A84B03EB4212927F2AB303EBA1
:10B9D00046139B7F934220D10027012329466D0106
:10B9E00006F80830022238466DB206F8097006F8EB
:10B9F0000A70FDF7D9FE45F0060140F2FF7201F032
:10BA0000E6013846FDF703FE45F00801D4F80320AF
:10BA100001F0E8013846FDF7FAFD0136032ECDD1DD
:10BA200005B0BDE8F08FB378022B00F24882DFF852
:10BA30004C82DFF84092DFF838A20026A278F5B2F7
:10BA4000AA4209D0884B03EB4212927F32B303EB38
:10BA500046139B7F934221D10027012329466D0184
:10BA600006F80830022238466DB206F8097006F86A
:10BA70000A70FDF799FE45F0060140F2FF7201F0F1
:10BA8000E6013846FDF7C3FDD4F8032045F0080170
:10BA9000524201F0E8013846FDF7B9FD0136032EA8
:10BAA000CCD1BDE7B378022B00F20982DFF8CC815C
:10BAB000DFF8BC916C4F0026A378F5B2AB4208D0FA
:10BAC00007EB43139B7FD3B107EB4612927F9A4259
:10BAD00015D1284603F014F9022229460020FDF76B
:10BAE00063FE690141F0080101F0E8010020FDF763
:10BAF00011FE012306F80830002306F8093001364C
:10BB0000032ED9D18CE7B078022803D97278022AA3
:10BB100040F0D5816278032A00F2BA81DFE812F0A2
:10BB200004003A0079008401DFF84481DFF8449191
:10BB30004E4F0025A278AA4209D04B4B03EB42128C
:10BB4000927F1AB303EB45139B7F93421ED1284685
:10BB5000FFF74EFD012303FA05F25FFA85FA3B7801
:10BB600000264FEA4A1123EA020301F0E001D4F86B
:10BB7000032005F80860304605F809603B70FDF7C2
:10BB800058FD324651463046FDF70EFE0135032D75
:10BB9000D0D145E7DFF8D4A00026A278B24209D080
:10BBA000314B03EB4212927F7AB303EB46139B7F38
:10BBB00093422AD13046FFF71BFD2D4B00275FFA39
:10BBC00086FBF7544FEA4B192A4B5FFA89F9F75471
:10BBD00049F002013846FDF7D9FF012202FA06F1C9
:10BBE000D4F803809AF80020804422EA01028AF8FF
:10BBF0000020494642463846FDF71BFD3A46594665
:10BC00003846FDF7D1FDC5F804800136032EC4D1B6
:10BC100006E7142B00F3538110F0C00630D1022840
:10BC200000F24D8103EB43030344134A0F4D52F8D6
:10BC30002370FFF7DDFCA1780D4B5E540D4B5E5475
:10BC4000012303FA01F02B78490123EA00033A4665
:10BC5000304601F0E0012B70FDF7EBFC3246A17895
:10BC60003046FDF7A1FDDBE6C8CDFF1F29CDFF1F44
:10BC700050CDFF1FC0CDFF1FF8CEFF1FBCC6FF1F5A
:10BC8000402E40F09C800026019602960396324694
:10BC900040FA02F1C90706D504A931440136032E42
:10BCA00001F8102C02D00132032AF1D1DFF83C83D5
:10BCB000002703EB4309B7423DD1012F0BDD022FD3
:10BCC000019E029D55D1AE424EDD9DF801202946D0
:10BCD0003046FFF733FCC54FDFF81883DFF81893C1
:10BCE0000025A3782B41DA0721D5D4F80330C048CA
:10BCF00003EB43032B445FFA85FA57F82320012313
:10BD000003FA05F10378002623EA01034FEA4A11FA
:10BD1000037001F0E001304605F8086005F809609D
:10BD2000FDF787FC324651463046FDF73DFD0135B3
:10BD3000032DD6D174E61DF807502846FFF758FCAE
:10BD4000690141F0020101F0E20100204D44FDF7DC
:10BD50001DFF58F82520801A002801ABB8BF4042CB
:10BD600043F827000137A6E79DF800203146284612
:10BD7000AFE7AE42039F16DDBE4209DD9DF801200C
:10BD800029463046FFF7DAFB9DF8022039469FE747
:10BD90009DF8002031463846FFF7D0FB9DF8012082
:10BDA0002946384695E7BD4231469DF80020F2DD30
:10BDB0002846FFF7C3FB9DF802203946D7E7802EBF
:10BDC0007DD1DFF828928B4FDFF82C820025A378F5
:10BDD0002B41DB0724D5D4F8033003EB43032B447A
:10BDE000284659F823A0FFF703FC814A012303FAF0
:10BDF00005F113785FFA85FB002623EA01034FEA79
:10BE00004B11137001F0E00152463046EE5505F833
:10BE10000860FDF70EFC324659463046FDF7C4FC7B
:10BE20000135032DD3D1FBE5022848D8142B46DC7D
:10BE3000400140F0020101F0E2010020FDF7A6FE02
:10BE4000D4F80330A178694A03EB43030B4400267E
:10BE500052F8235005440846FFF7CAFBA178654B0A
:10BE600063485E54644B5E54012303FA01F2037885
:10BE7000490123EA020303702A46304601F0E0013B
:10BE8000FDF7D7FB3246A1783046FDF78DFCC7E5BC
:10BE900003232B70C4E5FEF767FBC1E573789A1F97
:10BEA000012A0AD98C2B08D0C02B06D0C72B04D06E
:10BEB00003F13402D2B2322A04D8A2782AB1042380
:10BEC0002B70ADE5B278022AF9D89A2B25D8992B98
:10BED00080F0A380822B7AD013D8062B6DD006D8A1
:10BEE000042B60D0052B63D003232B7098E5072B20
:10BEF0001ED00C3B012BF7D81421A078FDF76CFD68
:10BF00008EE58C2B68D003D8832B4CD0862BEAE7A8
:10BF10008D2B7DD0933B022BEDE7C72B4DD020D846
:10BF2000C12B00F089800DD8B52B7BD0C02BDBD185
:10BF3000A078324B03EB40134001997A4A30FDF769
:10BF40000BF96DE5C22B00F08180C32BCCD1A0781A
:10BF50002B4902304001042201441044FDF75BF9F3
:10BF60005EE5D42B00F085800DD8CC2B77D0D22B7A
:10BF7000BAD1A07823490230400101440422103094
:10BF8000FDF749F94CE5D62B00F087807BD3FE2BDB
:10BF9000AAD1A0781C4902304001014401220C3092
:10BFA000FDF739F93CE50621A078FDF715FD37E5E9
:10BFB0000C21A078FDF710FD32E5A0780F4B03EBC4
:10BFC00040134001597A4930FDF7C6F828E50421AD
:10BFD000A078FDF701FD23E5A378002B7FF46FAF78
:10BFE00001220A494B20FDF716F919E5F8CEFF1F8B
:10BFF00029CDFF1F50CDFF1FC0CDFF1FC8CDFF1F94
:10C000008CCDFF1F98CDFF1F94CDFF1FD3CDFF1FF9
:10C010001A21A078FDF7E0FC02E51821A078FDF7D1
:10C02000DBFCFDE4A078BF4902304001014404225A
:10C030001830FDF7F0F8F3E4A078BB4B03EB4013A6
:10C040004001197A4830FDF787F8E9E4A078B7494C
:10C050000230400104220144FDF7DDF8E0E4A0785D
:10C06000B34902304001014402220E30FDF7D3F8FB
:10C07000D6E4A078AF4902304001014404221430D4
:10C08000FDF7C9F8CCE4A078AB4902304001014487
:10C0900001221E30FDF7BFF8C2E4A078A7490230A4
:10C0A0004001014402221C30FDF7B5F8B8E4737872
:10C0B0009A1F012A0AD98C2B08D0C02B06D0C72B77
:10C0C00004D003F13402D2B2322A17D8A278002A5F
:10C0D0007FF4F5AE9A2B2DD8992B80F0D080822B4F
:10C0E00000F0AB8018D8062B00F09C800AD8042BF7
:10C0F00069D0052B7CD003232B7091E4B278022AFF
:10C10000E8D9DCE6072B21D00C3B012BF3D8142116
:10C11000A078FDF73DFC83E48C2B00F0948003D8DD
:10C12000832B50D0862BE5E78D2B00F0A280933B2C
:10C13000022BEBE7C72B75D021D8C12B00F0B080C4
:10C140000ED8B52B00F0A180C02BD4D1A47860010B
:10C150004A30FDF7DAF8744B03EB441398725FE44E
:10C16000C22B00F0A880C32BC5D1A078744902303F
:10C170004001042201441044FDF7E0F850E4D42BC0
:10C1800000F0AE800ED8CC2B00F09F80D22BB2D125
:10C19000A0786C4902304001014404221030FDF7C0
:10C1A000CDF83DE4D62B00F0B180C0F0A480FE2B8A
:10C1B000A1D1A078644902304001014401220C3031
:10C1C000FDF7BCF82CE40621A078FDF7E1FBA5788B
:10C1D000690141F0060101F0E6010020FDF7CEFA09
:10C1E0005A4B5B4A43F82500A3780021D15417E449
:10C1F000A0780C21FDF7CCFBA578690141F00C017A
:10C2000001F0EC010020FDF7B9FA524B504A43F817
:10C210002500A0780021115453F82010FDF72BFBC6
:10C22000FFF7FEBBA47860014930FDF76EF83E4B86
:10C2300003EB44135872FFF7F3BB0421A078FDF71A
:10C24000A7FBFFF7EDBBA378002B7FF438AE364D8C
:10C25000012205F10B014B20FDF770F8A07805EBEA
:10C260004015E97AC1F10801C9B2FDF70BFFFFF7EC
:10C27000D7BB1A21A078FDF78BFBFFF7D1BB1821A4
:10C28000A078FDF785FBFFF7CBBBA07825490230EE
:10C290004001014404221830FDF750F8FFF7C0BBFD
:10C2A000A47860014830FDF730F81F4B03EB4413CE
:10C2B0001872FFF7B5BBA0781C4902304001042278
:10C2C0000144FDF73BF8FFF7ABBBA07818490230FB
:10C2D0004001014402220E30FDF730F8FFF7A0BB09
:10C2E000A078144902304001014404221430FDF7C3
:10C2F00025F8FFF795BBA0780F49023040010144B3
:10C3000001221E30FDF71AF8FFF78ABBA0780B490F
:10C3100002304001014402221C30FDF70FF8FFF704
:10C320007FBB00BFA0CDFF1FC8CDFF1F88CDFF1F63
:10C3300096CDFF1F9CCDFF1FA6CDFF1FA4CDFF1FD5
:10C340008CCDFF1F98CDFF1F94CDFF1F20D4FF1F62
:10C35000BCC6FF1F14D0FF1FB378022B00F0B480BF
:10C36000032B00F0B680002B40F04B817378502BEC
:10C3700000F0818024D8472B6DD011D8422B61D09A
:10C3800006D8402B43D0412B58D003232B7043E0D9
:10C39000452B5AD05CD8442BF7D1A84BDB694FE032
:10C3A0004C2B61D006D8492B58D04B2BEDD1A34B49
:10C3B000DB7845E04E2BA14B5BD058D95B7E3FE04C
:10C3C000802B67D012D8532B5BD006D8512B55D079
:10C3D000522BDAD1994B1B6A32E0552B57D053D3ED
:10C3E000562BD2D1954B93F8243029E0832B5AD089
:10C3F00005D8812B51D0822BC7D1914BCEE7852B0D
:10C4000057D053D3FF2BC0D18E4B1B7828E040F27E
:10C41000FF70FCF77AFF68608B4B1B78002B3FF4B2
:10C42000FFAA8A4B6A681A60894B002A40F0EB80A9
:10C430001A6842F008021A60FFF7F2BA7F4B1B78C5
:10C440006B60E9E77D4B5B78FAE77C4B5B79F7E75C
:10C450007A4BDB68F4E7794B9B68F1E7774BDB7D40
:10C46000003318BF0123EBE7744B9B78E8E75B7D53
:10C47000E6E7DB8CE4E7714B9B7DE1E76F4B1B7DCF
:10C48000DEE76E4B1B69DBE76C4B9B7ED8E76B4BA3
:10C49000DB7ED5E76A4B1B7ED2E7694B1B7E1E1FF6
:10C4A00073427341CCE7664B5B68C9E7694B1B6815
:10C4B000C6E7634A6848936843F2390100FB0313F7
:10C4C000936023F00043BBE77278644B53F822304B
:10C4D000B6E773782E2B3FF658AF01A252F823F03F
:10C4E0009DC50000A1C50000A5C500008BC30000CC
:10C4F0008BC300008BC300008BC300008BC3000004
:10C500008BC30000A9C50000ADC50000B1C5000087
:10C510008BC300008BC300008BC300008BC30000E3
:10C520008BC300008BC300008BC300008BC30000D3
:10C530008BC300008BC300008BC300008BC30000C3
:10C540008BC300008BC300008BC30000B7C5000085
:10C55000BFC50000C7C50000CBC50000CFC50000A7
:10C56000D3C500008BC300008BC300008BC3000049
:10C570008BC300008BC300008BC30000D7C5000035
:10C58000DDC50000E1C50000E5C50000EBC5000009
:10C59000F1C50000F7C50000FDC50000304B86E77F
:10C5A0002F4B81E72E4B57E72D4B52E72C4B69E77A
:10C5B0002B4B5B6944E70020FDF79BFA2BE700203B
:10C5C000FDF7ACFA27E70120F6E70120F8E70220A3
:10C5D000F2E70220F4E7224B9B6931E7204BDDE6CE
:10C5E0001F4BF8E61E4B5B6A2AE71D4B9B6A27E749
:10C5F0001B4BDB6A24E71A4B1B6B21E7184B5B6B69
:10C600001EE70423C2E61A6822F008021A60FFF748
:10C6100007BAB378022B27D17078372809D800F5EC
:10C62000A7701049800004220144FCF7F4FDFFF7D5
:10C63000F7B903232B70FFF7F3B900BF0CC0FF1F3E
:10C64000BCC6FF1F02D0FF1F03D0FF1FF4CFFF1F88
:10C65000F4CEFF1F04D0FF1F6D4EC64120D0FF1F38
:10C6600038CEFF1FE8CAFF1F04233B70FFF7D8B97D
:10C67000B378022B0CD170783728DAD800F5A77080
:10C68000A149800004220144FCF758FEFFF7C8B915
:10C6900004233B70FFF7C4B902F02AFBFFF7C0B9CF
:10C6A00002F02EFBFFF7BCB902F032FB974B78602B
:10C6B0001B78002B3FF4B4A9954B1860954B1A6872
:10C6C00020B942F008021A60FFF7AAB922F0080266
:10C6D0001A60FFF7A5B9B2782AB1022A0CD0042358
:10C6E0003B70FFF79DB97278002A7FF499A918462C
:10C6F000FCF70CFBFFF794B97078072808D81BB932
:10C70000FCF7EAF9FFF78CB9FCF7C2F9FFF788B933
:10C71000FF287FF485A95D1C0ABF7D4BD8B218782D
:10C72000FCF7FEF9FFF77CB9B378012B25D023B1D4
:10C73000022B26D004233B700AE07078082803D827
:10C74000FCF7FFF9686003E00A2811D100237B6041
:10C750006E4B1B78002B3FF463A96D4B6A681A601F
:10C760006C4B92B91A6842F008021A60FFF758B988
:10C77000FF28EDD1FCF750FAE4E7707802F012FBE5
:10C78000E0E77078FCF712FADCE71A6822F008029A
:10C790001A60FFF745B910681844106012685D4BC5
:10C7A00012BB1A6842F008021A60FFF739B9106824
:10C7B000C01AF2E710685843EFE7106890FBF3F0F7
:10C7C000EBE7116891FBF3F003FB10131360E5E74F
:10C7D00010681840E1E710681843DEE71068584019
:10C7E000DBE71368DB43F1E71A6822F008021A60FE
:10C7F000FFF716B9464A1168464A8B4213680BDAAE
:10C8000023F0030343F004031360136871B943F08A
:10C8100008031360FFF704B90BBF23F0060323F0EE
:10C82000050343F0010343F00203EDE723F008039F
:10C830001360FFF7F5B872780C2A3FF6F1A8DFE82D
:10C8400002F0071019222B343E4750596D767F00B5
:10C85000304A126814077FF5E3A82F4AD361FFF727
:10C86000DFB82C4A126810073FF5DAA82A4AD361CC
:10C87000FFF7D6B8274A1268D1077FF5D1A8264A14
:10C88000D361FFF7CDB8234A1268D2073FF5C8A895
:10C89000214AD361FFF7C4B81E4A126857077FF5D3
:10C8A000BFA81D4AD361FFF7BBB81A4A126812F03D
:10C8B000050F3FF4B5A8184AD361FFF7B1B8154A80
:10C8C000126896077FF5ACA8134AD361FFF7A8B8A2
:10C8D000104A126895073FF4A3A80F4AD361FFF7E7
:10C8E0009FB80C4A1268D4067FF59AA80A4AD36109
:10C8F000FFF796B8074A126890067FF591A8064A96
:10C90000D361FFF78DB800BFE8CAFF1F03D0FF1F38
:10C91000F4CFFF1FF4CEFF1FBCC6FF1FB44A12683E
:10C9200051067FF57DA8B34AD361FFF779B8B04AC5
:10C93000126812067FF574A8AE4AD361FFF770B88B
:10C94000AB4A1268D7057FF56BA8AA4AD361FFF7F7
:10C9500067B8A84AD361FFF763B8A64A136A002BE9
:10C960003FF45EA8013B136202EB83035B6AD36171
:10C97000FFF756B873782E2B04D89F4A0121D15463
:10C98000FFF74EB8FF2B7FF454AE9A4B012283F889
:10C990004420FFF745B873782E2B04D8964A00211F
:10C9A000D154FFF73DB8FF2B7FF443AE914B0022EB
:10C9B00083F84420FFF734B8FBF7ACFEEB6CC01AE9
:10C9C0000028AB6CB8BF4042984295BFEB6900238A
:10C9D00003F1FF3385F8453098BFEB61FFF720B8CE
:10C9E000A07802F095F940B9814A85F845001368AE
:10C9F00023F010031360FFF713B8AB6C9BB1FBF788
:10CA000089FEEB6CC01A0028AB6CB8BF404298425C
:10CA100009D9774A002385F84530136843F010039D
:10CA20001360FEF7FDBFEB69013BEB61FEF7F8BF5A
:10CA30000020FCF786FEA3785B00184110F001048B
:10CA400009D06B4A002385F84530136823F01003A2
:10CA50001360FEF7E5BFAB6C93B1FBF75BFEEB6CCD
:10CA6000C01A0028AB6CB8BF4042984208D9604A4F
:10CA700085F84540136843F010031360FEF7D0BFFC
:10CA8000EB69013BEB61FEF7CBBF01AA7C210020E3
:10CA9000FCF75DFEA3789DF806405A000223934000
:10CAA0001C4009D0524A002385F84530136823F012
:10CAB00010031360FEF7B4BFAB6C93B1FBF72AFE13
:10CAC000EB6CC01A0028AB6CB8BF4042984208D942
:10CAD000474A85F84540136843F010031360FEF79A
:10CAE0009FBFEB69013BEB61FEF79ABF01AA7C2176
:10CAF0000020FCF72CFEA2789DF80630520013416E
:10CB000013F0010409D03A4A002385F84530136830
:10CB100023F010031360FEF783BFAB6C93B1FBF7F8
:10CB2000F9FDEB6CC01A0028AB6CB8BF40429842CC
:10CB300008D92F4A85F84540136843F01003136065
:10CB4000FEF76EBFEB69013BEB61FEF769BF294B56
:10CB500000221A76FEF764BFFF287FF4B0A9274EA3
:10CB60003AB300254FF003080C27607818FB0051FA
:10CB70000138784300F5C36000EB8500042206EB22
:10CB800081010135FCF747FB032DEED1FEF748BFCD
:10CB900029197819042231440435FCF73CFB0C2D8B
:10CBA000F6D10C34FC2C3EF43BAF002504F20C67AC
:10CBB000EEE70C24F9E77378142B3FF63AADB27820
:10CBC000022A27D803EB430313440C4A52F82320CC
:10CBD0000B4B7A601B78002B3EF422AF094B1A6096
:10CBE000034B8AB91A6842F008021A60FEF718BFB0
:10CBF000F4CEFF1FBCC6FF1F8ACEFF1FF8CEFF1F5B
:10CC000003D0FF1FF4CFFF1F1A6822F008021A603A
:10CC1000FEF706BFFF2A7FF452A9AD4E3BB30025B5
:10CC20004FF003080C27607818FB00510138784357
:10CC300000F5C36000EB8500042206EB810101359D
:10CC4000FCF77CFB032DEED1FEF7EABE291978191B
:10CC5000042231440435FCF771FB0C2DF6D10C3461
:10CC6000FC2C3EF4DDAE002504F20C67EEE70C244C
:10CC7000F9E77678142E3FF6DCACA77838062ED587
:10CC8000934FDFF850820025A3782B41D9070DD5AB
:10CC90006901667841F0020101F0E2010020FCF731
:10CCA00075FF06EB46062E4447F8260098F81A3022
:10CCB00083B1637873B1032111FB03510C20013B55
:10CCC000584300F5C360042207EB810100EB8500A7
:10CCD000FCF7A1FA0135032DD6D1FEF7A1BE022F34
:10CCE0003FF6EDA8790141F0020101F0E2010020D8
:10CCF000FCF74CFF774B764D9B7E06EB46063E4499
:10CD000045F82600002B3EF48BAE6278002A3EF4F4
:10CD100087AEA078032111FB02010C23013A534393
:10CD200003F5C363042205EB810102FB0030FCF72D
:10CD300072FAFEF775BE7278674B0A2A0CD8DFE8E4
:10CD400002F006151A1F252D32373C414500634974
:10CD50001A6809680A441A601A68614B002A3AD1B5
:10CD60001A6842F008021A60FEF75ABE5B491A6858
:10CD70000968521AEFE7594A196812684A43EAE704
:10CD800056491A68096892FBF1F2E4E7534A1868B9
:10CD9000116890FBF1F201FB1202DCE74F491A68BF
:10CDA00009680A40D7E74D491A6809680A43D2E77B
:10CDB0004A491A6809684A40CDE748490A68D24397
:10CDC0000A60C9E71968454A1160C5E7434A19680E
:10CDD00010681860F8E71A6822F008021A60FEF777
:10CDE0001FBE3D4B1B68C6F80330FDF7BDFBFEF7C9
:10CDF00017BE7378052B3EF613AEDFE803F0030A87
:10CE000011181F26364A136803F00F031360FEF74C
:10CE100007BE334A136823F010031360FEF700BE09
:10CE20002F4A136823F020031360FEF7F9BD2C4A44
:10CE3000136823F040031360FEF7F2BD284A13681D
:10CE400023F080031360FEF7EBBD254A136823F43B
:10CE500080731360FEF7E4BD71782E293FF6E9ABCD
:10CE6000204A02EB81021365FEF7DABD1D4B1A4A18
:10CE7000D3F80C111160194AD3F810111160D3F8CE
:10CE80001421DA61164AD3F818111160D3F81C2165
:10CE900083F84520D3F82021DA64D3F824219A645A
:10CEA00093F82811104A505C08B101205054002218
:10CEB00083F82C21FEF7B4BD00F08CFEFEF7B0BD68
:10CEC00000F089FEFEF7ACBD00F098FEFEF7A8BDAD
:10CED000F8CEFF1F0CC0FF1FF4CFFF1F10D0FF1FA5
:10CEE000F4CEFF1FBCC6FF1F8ACEFF1F00F088FED6
:10CEF000FEF796BD00F085FEFEF792BD00F082FEC3
:10CF0000FEF78EBDA54B00221A76FEF789BD72781A
:10CF10002AB1012A08D003233B70FEF781BD9F4B45
:10CF200001221A76FEF77CBD40F2FE718B423EF67E
:10CF3000C6AF9A490A76CB61FEF772BD974A984808
:10CF4000002382F8443082F82C3102F150044FF073
:10CF5000FF35194644F82350C15401332F2BF9D122
:10CF6000904B11761960904BD16119608F4B116213
:10CF700082F845101960FEF753BD127D92070BD45D
:10CF800040F2FE7293423EF69AAF844A0421117633
:10CF9000C2F83031FEF744BD08233B70FEF740BDB8
:10CFA0007E4B00221A76FEF73BBD2B460022E25450
:10CFB0000133082BFBD123782372FEF731BD737840
:10CFC000012B19D005D3022B1FD003233B70FEF792
:10CFD00027BD774B01221A70764B774A9B781370E6
:10CFE000764B196800230139013311F8010FD05431
:10CFF000082BF9D1FEF714BD0422FA717B71562279
:10D000000923BA713B71FEF70BBD694B6C480122D5
:10D010001A70684B684A9B78137000230133191803
:10D02000082B11F8091CD154F8D1FEF7F9BC73781C
:10D03000032B3EF6F5ACDFE803F0020F1B20574B45
:10D040001A7EFA7193F84520D3F83031BA711A0A72
:10D050007A713B71FEF7E4BC504B1A7EFA7193F87B
:10D060004520DB69BA711A0A7A713B71FEF7D8BCA8
:10D070004C4B1B687B60FEF7D3BC4B4B1B687B6043
:10D08000FEF7CEBC7278002A7EF4CAACB1780029D3
:10D090007EF4C6AC40F2D24293427EF4C1AC40F280
:10D0A000FF70FCF759F8FBF7BEFF0120FBF70EFC01
:10D0B000FEF7B6BC0122FEF734BC74782CB1012C0B
:10D0C00014D003233B70FEF7ABBC04220DEB02012E
:10D0D00040F2FB70FCF732F9019BD6F803209A422C
:10D0E00006BF01237B607C60FEF79ABCB3782A2BD5
:10D0F00007D10422334940F2FB70FCF78CF8FEF7AD
:10D100008FBC03233B70FEF78BBC244CD4F8380152
:10D11000002104F59E7281423EF482AC52F8215007
:10D120009D4201F1010520D102EB8503043B01384A
:10D13000814214D3C4F83801FEF772BC174AD2F802
:10D14000381109299DBF481CC2F8380102EB810241
:10D15000092394BFC2F83C313B70FEF761BC53F821
:10D16000042F43F8042C0131E2E72946D3E70B4AA8
:10D170000023C2F83831194602F59E7242F8231096
:10D1800001330A2BFAD1FEF74BBC0A237B60FEF772
:10D1900047BC03233B70FEF743BC00BFBCC6FF1F68
:10D1A0008ACEFF1FF4CFFF1F10D0FF1FF4CEFF1F4A
:10D1B000F8CFFF1F0CC0FF1FF9CFFF1F08C0FF1FD4
:10D1C00000800000EFCEFF1F7378812B7EF477AED6
:10D1D000B378922B7EF473AEB379A32B7EF46FAE4B
:10D1E0007379B42B7EF46BAE3379C52B7EF467AEC6
:10D1F000F378D62B7EF463AEFBF73FFEFBF78AFA9B
:10D200000446FBF787FA001B0028B8BF4042B0F580
:10D210007A7FF6DBFBF758FB134B00221A604FF0C6
:10D22000FF32C3F87021C3F87022C3F87421C3F829
:10D230007422C3F87821C3F87822C3F87C21C3F89C
:10D240007C220A4B0A4A1A600120FBF73FFBFEF7DB
:10D25000E7BB40F2D24293427EF4E2AB054B01229F
:10D2600083F86421FEF7DCBB10E000E000C0FF1F84
:10D2700078563412BCC6FF1F364B2DE9F047002408
:10D280001C60354B354D1C60354BDFF8E880354F61
:10D29000EC611C6085F845406601F6B246F0060177
:10D2A0000020FCF773FC46F00C0148F82400002035
:10D2B000FCF76CFC47F824000134032CECD12A4B1A
:10D2C000D97AC1F10801C9B20020FCF7DBFE274A78
:10D2D00000231946904642F823100133B3F5807FAE
:10D2E000F9D1234CA37E03BBE37E13B394F824103F
:10D2F0000020FCF79FFA637D4BB3FBF783FD30B34F
:10D3000001232B76BDE8F087B91909EB0700042249
:10D3100051440437FCF712F80C2FF5D10C36FC2ED3
:10D32000E2D0002706F20C69EEE70C26DFF848A0F1
:10D33000F7E74FF4A766A6F5A761304604224144FB
:10D340000436FBF7FBFFB6F5C36FF4D1CEE700233D
:10D35000D7E700BFF4CFFF1F10D0FF1FBCC6FF1FD1
:10D36000F4CEFF1F14D0FF1FC8CDFF1F20D0FF1F1A
:10D370000CC0FF1F20D4FF1FF8CEFF1FF7B50F4CC6
:10D3800007460E4694E803008DE803000C49C1F8F7
:10D3900003300C4B8A7000220F704E701A70FEF72B
:10D3A00047F9094A217882F865119DE8030063680E
:10D3B00084E80300184603B0F0BD00BF08D0FF1F8B
:10D3C000ECCEFF1F03D0FF1FBCC6FF1FF7B50446FE
:10D3D0001F4A63781370A3785370E37893702379AE
:10D3E000937163795371A3791A4D1371E379D370F3
:10D3F0000E4695E80300184B00221A708DE80300D2
:10D40000FEF716F9154B1A786F462B469AB932700B
:10D4100072702A78B2706A78F270EA793271AA79F9
:10D4200072716A79B2712A79F27197E8030083E820
:10D43000030003B0F0BD012AF7D10948721EF11DA7
:10D4400010F8014F02F8014F8A42F9D1EDE700BF11
:10D45000ECCEFF1F08D0FF1F03D0FF1FF8CFFF1F28
:10D46000F9CFFF1F014B93F865017047BCC6FF1F42
:10D470002DE9F043994B9A4C1B788FB06BB1994BC7
:10D480001B78063BDBB2192B04D8974A22FA03F328
:10D49000D90702D4002384F8343194F83431934E00
:10D4A0005A1E012A51D89249012BCA68079214BF0B
:10D4B000082307238DF81830327894F866318DF8F8
:10D4C000193000238DF81A30002A33D18B688DF87B
:10D4D0002030884B8DF8272019788DF82110597845
:10D4E0008DF82210D9798DF8231099798DF82410B0
:10D4F00059791B798DF825108DF8263006A801F092
:10D5000071FD002800F016837B4B1A789846002A9C
:10D5100000F01E81794B7A4F1B78013B062B00F2FD
:10D520001381DFE813F0F100F1005701110111013F
:10D5300011017E01012AE1D17248013306AA1A4481
:10D54000195CD171082BF8D1D8E7032B3DD1337882
:10D5500083BBDFF89C81674F98F8020098F8015070
:10D560003B7805441D447B781D44FB791D44BB7901
:10D570001D447B791D443B791D44FBF705F998F860
:10D580000100FBF701F93878FBF7FEF87878FBF734
:10D59000FBF8F879FBF7F8F8B879FBF7F5F8787944
:10D5A000FBF7F2F83879EDB2FBF7EEF82846FBF717
:10D5B000EBF8A9E7012BA7D1524F0025785D013583
:10D5C000FBF7E2F8092DF9D19EE7042B2BD1484F48
:10D5D000DFF82081B8787D780023012205441544C6
:10D5E00088F8013088F80020C8F80430FBF7CCF840
:10D5F0007878FBF7C9F898F80000FBF7C5F898F8B9
:10D600000100FBF7C1F898F80700FBF7BDF898F8A0
:10D610000600FBF7B9F898F80500FBF7B5F8EDB28E
:10D6200098F80400C0E7072B37D1337853BB304B51
:10D630009F7893F801802F4B8DF800701D785878F3
:10D64000D9798DF8025047443D449A798DF803000A
:10D65000284493F805C08DF80410014493F804E0C1
:10D660008DF805200A440CEB020373448DF8018009
:10D670008DF806C08DF807E08DF808306846FBF796
:10D68000F9FB41E7012BF9D11E4900235A5C0DF843
:10D6900003200133092BF9D1F0E7082B7FF434AFD5
:10D6A000144A1349002301205370107053608A7884
:10D6B00049788DF800200A4402448DF801108DF855
:10D6C00002008DF803308DF804308DF805308DF8A8
:10D6D00006308DF807308DF80820CFE702D0FF1F05
:10D6E000BCC6FF1FECCEFF1F11020002F8CFFF1FC8
:10D6F0000CC0FF1F08D0FF1FB9CEFF1F80CEFF1F39
:10D7000053CDFF1FF9CFFF1FAA4A397893688DF8D0
:10D71000303080238DF831308A238DF83230002369
:10D720008DF833308DF834308DF835308DF8361073
:10D730008DF8293007218DF82A300AA8D3688DF892
:10D7400028100B9301F04EFC00233B7088F800304A
:10D75000002384F83431337094F8643113B101201C
:10D76000FBF7B4F806A801F0C9FB0646002800F054
:10D770003981914B9DF820201A709DF821205A7014
:10D780009DF822209A709DF823209A719DF82420FC
:10D790005A719DF825201A719DF82620DA709DF89F
:10D7A000193084F86631FAF7B5FF844B1860844B62
:10D7B00000221A709DF81830072B0CBF012302239A
:10D7C00084F83431237E5A1E012A4AD9052B48D0C9
:10D7D000012247E0DFF8DC913B7899F8020099F8E4
:10D7E000015005440A351D44FAF7CEFF99F80100AF
:10D7F000FAF7CAFF8020FAF7C7FF8A20FAF7C4FFBA
:10D800000020FAF7C1FF0020FAF7BEFF0020FAF768
:10D81000BBFFEDB23878FAF7B7FF2846FAF7B4FF46
:10D8200092E7644A507893788DF80C303A788DF806
:10D830000D00802103448DF80E100A338A218DF8E3
:10D840000F101344002103A88DF810108DF811104B
:10D850008DF812108DF813208DF81430FBF70AFBA9
:10D8600072E70022574B1A70237E042B04D1524BCF
:10D8700019780A0640F1618194F83421082A04D805
:10D8800040F25113D340DF0701D4FDF7D1FE94F8E5
:10D890003431092B6DD1FAF73DFFE3684A4DC01AC8
:10D8A00000282A68B8BF4042904208D9474B1A78EE
:10D8B000012A04BF02221A70FAF72CFFE060FAF77F
:10D8C00029FF23696A68C01A0028B8BF4042904205
:10D8D00008D93E4B5A78012A04BF02225A70FAF73F
:10D8E00019FF2061FAF716FF6369AA68C01A0028B9
:10D8F000B8BF4042904208D9344B9A78012A04BFFD
:10D9000002229A70FAF706FF606194F8443083B3FC
:10D9100094F82C316BBB2D4A2D481D46D15C022951
:10D9200040F0FF8050F823104E1C00F0F980294A87
:10D9300084F828311268C4F80C21274A1268C4F808
:10D940001021E269C4F81421244AE1611268C4F884
:10D95000182194F84520C4F81C210023E26CC4F877
:10D96000202184F84530A26CC4F82421012384F8D6
:10D970002C3194F83431092B04D1227E022A04BFC1
:10D9800005222276D4F83821002A00F0D380092B12
:10D9900040F0D080237E012B40F0CC80E16910481C
:10D9A000002350F823508D4240F0C0800523237699
:10D9B000C0E000BF0CC0FF1FECCEFF1F70CEFF1FEA
:10D9C00018CDFF1F03D0FF1F38CEFF1F8ACEFF1FC9
:10D9D0000CC7FF1FF4CFFF1F10D0FF1FF4CEFF1F97
:10D9E000F8C7FF1F03A8FAF7E7FE054600284ED048
:10D9F000FAF7FAFE08B184F8676194F867219DF898
:10DA00000C10531CDBB22244092B84F8673182F8D6
:10DA100068117FF429AF5E4A94F8681152780023A8
:10DA2000914284F867317FF41FAF5A495A5C013341
:10DA30001644082BF6B2F9D194F87031B34222D1D2
:10DA4000554B94F869211A7094F86A215A7094F829
:10DA50006B219A7094F86C219A7194F86D215A7127
:10DA600094F86E211A7194F86F21DA70FAF752FE69
:10DA70004A4B4B4A186000231370032284F8342168
:10DA800084F867319EE6042384F83431ECE60AAE6C
:10DA90003046FBF7DCF948B32B46F25C0133154402
:10DAA000082BEDB2F9D19DF83020AA42ECD13A4BC7
:10DAB0009DF829201A709DF82A205A709DF82B2075
:10DAC0009A709DF82C209A719DF82D205A719DF81E
:10DAD0002E201A719DF82F20DA70FAF71BFE2F4BBB
:10DAE00018602F4B00221A70072369E6237E013B42
:10DAF000012B3FF6B9AEE26940F2FE739A420CD8B0
:10DB0000FBF780F948B1E0692349431CE361FBF767
:10DB100049FA092384F834315AE600232376A3E630
:10DB2000D55401332F2B7FF4F9AE22E701339A420B
:10DB30007FF437AF0FB0BDE8F08394F834010828C4
:10DB400004D840F25112C240D207F3D4154DD3F895
:10DB50000330D4F830016B6040F2FE739842697074
:10DB600012D80D49FBF72EFB0B49D4F83001FBF717
:10DB70009BFA38B1D4F830310133C4F83031652321
:10DB80002B70D7E70723FBE707232B7000230EE753
:10DB90000CC0FF1F24C8FF1FECCEFF1F78CEFF1F55
:10DBA0007FCEFF1F08D0FF1F704710B5074CFAF754
:10DBB000B1FD2368C01AB0F5FA7F05D9044B2022C5
:10DBC000DA60FAF7A7FD206010BD00BF2CD4FF1F5C
:10DBD00000F00F407047064B5A7832B9D3F8031063
:10DBE000044B01B901221A7070470322024BFAE775
:10DBF000ECCEFF1F4CCDFF1F08D0FF1F70477047B2
:10DC000070477047704770472DE9F04F9E4C23785E
:10DC100085B033B96FF000436360A360E360012314
:10DC20002370257CDFF8A0824DB9E8B2FAF789FFAE
:10DC300008F805000135082DF7D101232374DFF81A
:10DC40008CA2924F272500264FF00209F0B2FAF776
:10DC500078FF18F80630834216D0B31D08F8060086
:10DC60005AF82330022B0AD0032B02D0012B0BD100
:10DC700050B17B5D012B08BF07F8059004E018B98F
:10DC80007A5D012A00D17B550136082E05F1010588
:10DC9000DCD17F4DEB69C3B17E4E3778AFB9FAF76F
:10DCA00039FD7D4B1B68C01A0028EB69B8BF4042A4
:10DCB00098420AD93846FBF7B3FE0120FBF7B0FEC5
:10DCC0000220FBF7ADFE012333702B6AC3B1734E04
:10DCD0003778AFB9FAF71EFD714B1B68C01A0028E0
:10DCE0002B6AB8BF404298420AD93846FBF798FEE3
:10DCF0000120FBF795FE0220FBF792FE0123337013
:10DD0000684D2B7B002B40F0B482FAF703FDE369EA
:10DD1000C01A0028B8BF40420A2804DC624B1B69C5
:10DD2000DF0700F1258294F82000002840F04781A9
:10DD30000A21FBF723FD074694F820005B4EFBF712
:10DD4000AFFF002F40D194F82010490141F00801A5
:10DD500001F0E8013846FBF711FDA8BBFAF7DAFC41
:10DD600094F8202004EB820305EB42115B68B1F8C4
:10DD70001CE0C01A00284FF00A03B8BF404203FB62
:10DD80000EF3984208DD897A1046FAF7ADFD94F853
:10DD900020300121464AD15494F8200087EAE778E0
:10DDA00056F83030A8EBE77898452BD2FCF76AFAA2
:10DDB00094F8203006EBC306727982422BD1002101
:10DDC0001846FCF72DFA26E094F8200087EAE7725F
:10DDD00056F83030A2EBE7729A4235BF06EBC0032B
:10DDE00005EB40131979597AFAF77EFD94F82080F3
:10DDF000FAF790FC04EB880894F82030C8F8040087
:10DE00000021C7E7FCF73EFA94F8203006EBC30682
:10DE100071798842D4D194F82000264B03440193B1
:10DE2000254B03440093254B002203EB800311464E
:10DE3000FCF7FAFA94F8200005EB40139B69BBB19C
:10DE4000FAF79EFFA0B194F8200005EB40139B6900
:10DE500098450DD9FBF7E4FD94F82030184A0121CC
:10DE6000D1540F33094AD15C012904BF0221D15496
:10DE700077B394F82060134B9B5DABBBFAF74AFC79
:10DE800004EB8606706255E030C8FF1F8ACEFF1F84
:10DE90000CC0FF1F7FCEFF1F78CEFF1F18CDFF1FC6
:10DEA00070CEFF1FC8CDFF1FC0F00F4034CDFF1F45
:10DEB00081CEFF1FC3CDFF1F30CDFF1F58CDFF1FE9
:10DEC000C0CDFF1F84CEFF1F41C8FF1F38CEFF1FEC
:10DED00094F82010490141F0080101F0E8013846AA
:10DEE000FBF74CFC0028C4D194F8203005EB43121A
:10DEF000D28912B9AA4AD35CE3B1FAF70BFC94F8C1
:10DF0000202004EB82035B6AC01A05EB4213002851
:10DF1000D9894FF00A03B8BF40424B43984209DD0C
:10DF2000A04EB35C33B91046FCF7EAFA94F82030FF
:10DF30000122F25494F8202051016B185B69002BE8
:10DF40003DD0994B9E5C9846CEBBC7B341F00201D1
:10DF500001F0E2013046FBF719FE074694F8200075
:10DF600001F00EF994F8201005EB4113381A5B69A3
:10DF7000002883EAE372B8BF4042A2EBE37290420A
:10DF80001DDD002B40F31E810846FBF749FD94F888
:10DF9000203005EB43139B7F002B40F0EC8094F87E
:10DFA0002030824A1533D15C012901D10221D1549C
:10DFB00094F82000012308F8003000F0A1FE0020B2
:10DFC000FBF7BFFB94F830308DF8080003F0F8033E
:10DFD000C60748BF43F0010384F83030450748BF07
:10DFE00094F83030DFF8D8A144BF43F0020384F83E
:10DFF0003030C00648BF94F830309AF800C044BFB3
:10E0000043F0040384F83030694B94F830001978F9
:10E01000684B1E78684B1D78684B93F8009000237E
:10E020001F469E4698461A464CFA02FB1BF0010F0B
:10E0300040F002810132032AF6D1B8F1000F01D07D
:10E040008AF800C0BEF1000F01D0594A11700FB11B
:10E05000584A16700BB1584B1D70C10709D594F87A
:10E060003130DA0705D4514BDA78012A04BF022295
:10E07000DA70830709D594F831309F0705D44B4BEC
:10E080001A79012A04BF02221A71460709D594F8A9
:10E0900031305D0705D4454B5A79012A04BF02226D
:10E0A0005A7104AA94F8201084F831000323B1FBBC
:10E0B000F3F3134413F9083C002B49DA490141F00A
:10E0C000160103AA01F0F6010020FBF740FB9DF8C2
:10E0D0000E3058060AD594F8202002201B2110FB90
:10E0E000021232498D5C012D08BF885419060AD5E9
:10E0F00094F820202D490E3211F81200012804BF97
:10E10000022001F81200DA060AD594F82020022035
:10E110001B2110FB021225498D5C012D08BF88547C
:10E120009B060AD594F82030204A0E3312F81310BB
:10E13000012904BF022102F8131094F820104901AC
:10E1400041F0160103AA01F0F6010020FBF73AFAAC
:10E1500094F8200000F002F994F820300133DBB28B
:10E16000032B88BF002384F82030FAF7D3FAE0614C
:10E1700005B0BDE8F08F94F8202005EB461305EBC1
:10E1800042129B7F927F9A4205D13046FBF748FCB2
:10E19000F0B200F0B5FD0136032EECD1FFE600BF72
:10E1A00084CEFF1F87CEFF1F50CDFF1F8ACEFF1FDB
:10E1B00029CDFF1F53CDFF1FB9CEFF1F28CDFF1F55
:10E1C00054CDFF1F02223046FBF7EEFA94F82010E0
:10E1D000490141F0080101F0E8013046FBF79AFAE5
:10E1E00094F8203005EB43139B7F002B3FF4E0AE07
:10E1F00094F8202005EB461305EB42129B7F927F9B
:10E200009A4210D1F7B2022239460020FBF7CCFA2D
:10E21000790141F00801002001F0E801FBF77AFAEA
:10E22000384600F06DFD0136032EE1D1C0E6012332
:10E230001D461F469E46FDE640FA02FB1BF0010FFD
:10E240003FF4F8AE41FA02FB1BF0010F7FF4F2AE8F
:10E25000012393405BB219431E43C9B2F6B2B9F130
:10E26000000FE4D10123CC461D461F469E4698462A
:10E27000E0E60022354E364B84F820201046019609
:10E2800000931146334BFCF7CFF894F82000335637
:10E29000314E002B04EB000393F832301CDB022BD1
:10E2A00001D1335C83B105EB4015697AFAF71CFBA9
:10E2B00094F82000FCF72EF994F82030E21802219F
:10E2C00082F832100022F25494F82050FAF722FA21
:10E2D00004EB850460604BE7012B1DD194F82030DE
:10E2E000F35C002B3FF444AF94F8200005EB40139F
:10E2F000997AFAF7F9FA94F8200005EB4015AB7A11
:10E30000F3B9FCF7FDF894F820301C44012284F89E
:10E3100032200022F2542BE7FAF7FCF994F820207F
:10E3200004EB820305EB42125B68928BC01A002853
:10E330004FF00A03B8BF404253439842CEDDD3E7C3
:10E34000335C002BDFD0FCF7E5F8DCE7C3CDFF1F23
:10E3500030CDFF1F58CDFF1F7CCEFF1F2DE9F04FA2
:10E3600046014FFA86FB85B04BF07C01044603AAB8
:10E3700001F0FC010020FBF7EAF94FEA44099DF99E
:10E380000EA0A64D0222012303FA09F302FA09F2B4
:10E390000AEA02020AEA030AAB19D2B21B7A009215
:10E3A00003F07F071B065FFA8AFA4FF0000013D5CF
:10E3B000FAF7C7FBB0FA80F35B09791E009A0729C8
:10E3C00000F28A82DFE811F00E000E000E000E004F
:10E3D0008B028B028B028B02FAF7B3FB031C18BF74
:10E3E0000123EAE78E490B5D88460F2B00F2748209
:10E3F000DFE813F07202100054007D008F00B800B7
:10E40000CF00F2001E016701CF01D40172021D028C
:10E41000480226024FF0000A5FFA8AFB5C4507D0EB
:10E42000AA19927F82B305EB4A11897F91422BD1C1
:10E430004FEA4B194FFA89F949F0140103AA01F088
:10E44000F4010020FBF783F949F00609754B9DF8AC
:10E450000D2043F82A205FFA89F949460020FBF78E
:10E460008DF9714B022243F82A0059460020FBF730
:10E470009BF940F2FF7249460020FBF7C8F80322DF
:10E4800059460020FBF7B3F90AF1010ABAF1030F6C
:10E49000C2D1023F012F38D8022337E008EB8403B2
:10E4A00021465A6802F0040242F001020020FBF704
:10E4B0009EF90027B9462E445FFA89F39C4205D0A5
:10E4C000B37F53B17A19927F9A4206D147F008017F
:10E4D0007A59C9B20020FBF79AF809F10109B9F19C
:10E4E000030F07F12007E7D108F80490F4E1BAF12F
:10E4F000000F00F0F1814BF0020101F0E201002079
:10E50000FBF744FB494B43F82400042308F804308C
:10E51000E2E108EB840321465A6802F0040242F06B
:10E5200002020020FBF763F90027B9462E445FFA88
:10E5300089F39C4205D0B37F5BB17A19927F9A42EE
:10E5400007D17A5947F008015242C9B20020FBF7BF
:10E550005EF809F10109B9F1030F07F12007E6D1CF
:10E560000523D3E7002A00F0B78100272E44FBB231
:10E57000A34206D0B37F3BB105EB4712927F9A428C
:10E5800002D13846FBF74CFA0137032FEFD10623AF
:10E59000BCE7032221460020FBF729F9DFF87C9035
:10E5A00000273544F9B28C4205D0AB7F6BB199F8A6
:10E5B0001E209A4209D1490141F00801D9F80420EE
:10E5C00001F0E8010020FBF722F80137032F09F1E1
:10E5D0002009E7D1072399E7002A40F07D810F4FFA
:10E5E000914635445FFA89F1A14204D0AB7F63B113
:10E5F000BA7F9A4209D17A68490141F00801524232
:10E6000001F0E8010020FBF702F809F10109B9F176
:10E61000030F07F12007E5D1082377E7C8CDFF1FD7
:10E6200068C8FF1F6CC8FF1F78C8FF1F1CCDFF1FE5
:10E63000002A00F051814BF0020101F0E2010020BC
:10E64000FBF7A4FABA4A52F8243000271B1A42F802
:10E6500024308346B946AB195FFA89F6B44205D037
:10E660009A7F2AB37919897F914221D14FFA87FA8B
:10E6700000224AF008011046C9B20093FAF7C7FF1A
:10E68000032231460020FBF7B2F87A194AF006015E
:10E690005268C9B20020FAF7BAFF5A46F9B2002010
:10E6A000FAF7C7FF002231461046FBF77DF8009BC2
:10E6B00009F10109B9F1030F07F12007CCD10923B2
:10E6C00024E70020FBF73DF840FA09F0C10740F1CC
:10E6D00003814FF00009AB19CA4600935FFA8AF331
:10E6E0009C4207D0009A927F0AB309EB0501897F0B
:10E6F00091421CD14FFA89FB00224BF008011046D1
:10E70000C9B20193FAF783FF019B02221946002048
:10E71000FBF74AF800224BF002011046C9B2FAF7A3
:10E7200088FF00225FFA89F11046FAF782FF0AF1AA
:10E73000010ABAF1030F09F12009CFD1033F012FDC
:10E740007CD8DFF8F4A14FF0000935445FFA89F76F
:10E75000BC4205D0AB7F9BB19AF81E209A420FD1E4
:10E76000022239460020FBF71FF8DAF8042079016D
:10E7700041F00801524201F0E8010020FAF747FF9A
:10E7800009F10109B9F1030F0AF1200ADED10A23C8
:10E79000BCE6002A00F0A0800B23B7E6002A40F078
:10E7A0009B804BF00201104601F0E2010092FBF762
:10E7B000EDF9009A8146174605EB060AF9B28C423C
:10E7C00007D09AF81E306BB105EB4712927F9A4240
:10E7D00008D1490141F00801002201F0E80110468A
:10E7E000FAF715FF0137032FE8D100272E44022343
:10E7F00099FBF3F95FFA87FA544506D0B37F8BB1E2
:10E8000005EB4712927F9A420CD14FEA4A114A46D1
:10E8100001F0E0010020FAF70CFF002251461046FB
:10E82000FAF7C2FF0137032FE4D10D236EE6002073
:10E83000FAF787FF40FA09F0C2074DD50E2365E6C7
:10E840004FF000092E445FFA89F7BC4206D0B37F2F
:10E8500093B105EB4912927F9A420DD102223946BB
:10E860000020FAF7A1FF790141F00801002201F030
:10E87000E8011046FAF7CBFE09F10109B9F1030FDF
:10E88000E1D1DBE7DFF8B4A000273B46AAF10C0B8F
:10E890005FFA87F94C4507D0AA19927FCAB105EBF8
:10E8A0004711897F914214D14FEA491141F0060185
:10E8B0005AF82720009301F0E6010020FAF7A7FE9E
:10E8C0001BF8272049460020FAF791FF009B08F823
:10E8D00007300137032FDBD105B0BDE8F08F1548B5
:10E8E000015D80460F29F7D801A050F821F000BF44
:10E8F000D9E8000041E90000BDE9000017EA000086
:10E9000037EA000093EA0000D9E80000A9EA000015
:10E91000D9E80000D9E8000063EB00007FEB0000BD
:10E9200005EB0000FDEB0000BDEC000079EC000001
:10E930001CCDFF1F68C8FF1FC8CDFF1F78C8FF1F71
:10E940004FF0000A5FFA8AFB5C4507D0AA19927F54
:10E9500042B305EB4A11897F914223D14FEA4B190B
:10E960004FFA89F949F0140103AA01F0F4010020DB
:10E97000FAF7EDFEBE4B9DF80D2043F82A205946CC
:10E9800002220020FAF710FF49F0060140F2FF7260
:10E9900001F0E6010020FAF73AFE03225946002072
:10E9A000FAF725FF0AF1010ABAF1030FCAD1062FBF
:10E9B0003FF472AD082F7FF4A8AD6DE5062F26D188
:10E9C00008EB84035A6802F0040242F00102214677
:10E9D0000020FAF70CFF0027B9462E445FFA89F3AE
:10E9E0009C4205D0B37F53B17A19927F9A4206D1E7
:10E9F00047F008017A59C9B20020FAF708FE09F178
:10EA00000109B9F1030F07F12007E7D16CE5082FE1
:10EA1000E1D10322DBE77A1F012A07D8BAF1000F00
:10EA200004D0062F3FF471AD0F236FE5002B3FF4A8
:10EA300053AF0C236AE5052F27D108EB84035A68EE
:10EA400002F0040242F0020221460020FAF7CFFE53
:10EA50000027B9462E445FFA89F39C4205D0B37F64
:10EA60005BB17A19927F9A4207D17A5947F008012F
:10EA70005242C9B20020FAF7CAFD09F10109B9F101
:10EA8000030F07F12007E6D16AE5072FE0D1032243
:10EA9000DAE7791F012903D812B1052FC4D1FBE4AD
:10EAA000002B7FF497AD17E7002B7FF415AF073FDE
:10EAB000012F0AD908EB84022146526802F00402B1
:10EAC00042F001021846FAF792FEDFF8A8910027FB
:10EAD0003544F9B28C4205D0AB7F6BB199F81E205A
:10EAE0009A4209D1490141F00801D9F8042001F006
:10EAF000E8010020FAF78BFD0137032F09F1200907
:10EB0000E7D144E6002B7FF4E7AE073F012F0AD997
:10EB100008EB84022146526802F0040242F002022D
:10EB20001846FAF764FEDFF84C9100273544F9B235
:10EB30008C4205D0AB7F73B199F81E209A420AD15E
:10EB4000D9F80420490141F00801524201F0E801DE
:10EB50000020FAF75CFD0137032F09F12009E6D107
:10EB600015E6002B3FF4B8AE4BF0020101F0E201D4
:10EB70000020FBF70BF808EB8403D8610CE6002BB0
:10EB80007FF4AAAE4BF00201184601F0E2010093B7
:10EB9000FAF7FCFF009BAA19824653731F46994659
:10EBA00008EB840B5FFA89F39C4206D0AA19927F86
:10EBB000E2B17919897F914218D17A1947F006019B
:10EBC00052680093C9B20020FAF733FDDBF81C202D
:10EBD00002210020524492FBF1F2F9B2FAF729FD2A
:10EBE000009B002219461046FAF7DEFD09F10109E3
:10EBF000B9F1030F07F12007D4D116E60020FAF788
:10EC0000A0FD40FA09F0C3077FF566AE0E2300278A
:10EC100008F80430B9462E445FFA89FA544505D005
:10EC2000B37FEBB17A19927F9A4219D14FFA87F8E4
:10EC3000002248F008011046C9B2FAF7E8FC0222A7
:10EC400051460020FAF7B0FD002248F002011046BC
:10EC5000C9B2FAF7EEFC0022F9B21046FAF7E9FC65
:10EC600009F10109B9F1030F07F12007D4D133E607
:10EC70006CC8FF1FC8CDFF1F4FF000092E445FFA7C
:10EC800089F7BC4206D0B37F93B105EB4912927F5E
:10EC90009A420DD1022239460020FAF785FD79010A
:10ECA00041F00801002201F0E8011046FAF7AFFC3C
:10ECB00009F10109B9F1030FE1D1BFE5DFF82C90AB
:10ECC00000272E44F9B28C4206D0B37F4BB105EB3E
:10ECD0004712927F9A4204D119F827200020FAF7B0
:10ECE00086FD0137032FEDD100230FE46CC8FF1F11
:10ECF000024B1A5C0AB901221A54704768C8FF1FF8
:10ED0000024B1A5C0AB10F221A54704768C8FF1FE1
:10ED1000014B185C704700BF68C8FF1F0E4B1A6894
:10ED200002F01F02052A0AD0062A0ED0042A10D1AA
:10ED30001A690A4992B20A8045221A6070471A6914
:10ED4000064992B28A804622F7E71A69034992B2CD
:10ED50004A804422F1E700BF00B00B4090C8FF1F7B
:10ED60000E4B41F230013A205A5842F000625A509C
:10ED700041F23C015A5842F000625A5003F5E82330
:10ED80000C229A6006491022DA6000225A620A6256
:10ED90004A628A6244221A6000F07ABA0070044023
:10EDA00000B0044009282BD8DFE800F0050A0D1058
:10EDB00014172A2A1A25134B1888C0F30B10704712
:10EDC000104B5888F9E70F4B9888F6E70D4B1888D9
:10EDD00080B270470B4B5888FAE70A4B9888F7E7E0
:10EDE000084B588883B24FF4987058434FF6FF731E
:10EDF00090FBF3F07047034B988883B23420F4E71C
:10EE00000020704790C8FF1F30B52E4D41F23C04E2
:10EE10002B5943F010032B512B4B4FF400749C647F
:10EE20006FF4F875DC64A3F51833A4F13E542C4458
:10EE30001C604FF400545C60244C1C601C68E401AE
:10EE4000FCD50138072834D8DFE800F0312F2D2B0E
:10EE5000293327041E4858601E4B002058631E4863
:10EE600018601E484FF0806400EA8145C3F8804076
:10EE7000C3F88450FAB100EA8240C3F89040C3F866
:10EE800094004FF08460C3F8A000C3F8A410AAB1A6
:10EE9000C3F8B000C3F8B42030BD1148DBE7114817
:10EEA000D9E71148D7E71148D5E71148D3E711480A
:10EEB000D1E71148CFE7C3F89020E2E7C3F8B020CC
:10EEC00030BD00BF0070044000A004400F0080501F
:10EED0008320FC01004002400F0080000000FC1F66
:10EEE0008720FE028720FE0B8720FE0E8720FE1D56
:10EEF0008720FE4A8720FE958720FE05384AD2F8F3
:10EF00008030C3F30363022B5FD0D2F89030C3F399
:10EF10000363022B5BD0D2F8A030C3F30363022B50
:10EF200006D0D2F8B030C3F30363022B56D10323CB
:10EF30001B0103F1402202F50032D2F88010C1F328
:10EF400003410170D2F8801011F4801118BF012123
:10EF50008170D2F8801011F4001118BF01214170A6
:10EF60004178B1BBD2F88410C1F38A4103F1402348
:10EF700003F500334160D3F88810090E0172D3F80D
:10EF80008810090C4172D3F88810090A8172D3F8ED
:10EF90008810C172D3F88C10090E0173D3F88C104D
:10EFA000090C4173D3F88C10090A8173D3F88C30A3
:10EFB000C373D2F880309B024CBF4FF084634FF094
:10EFC0008063C2F88030012070470023B0E701233E
:10EFD000AEE7D2F8841021F06041C7E70020704707
:10EFE00000400240184AD2F87031C3F303630C2B7F
:10EFF00010B527D04478436804B3C3F31103C2F8B3
:10F0000074318368104A1BBAC2F87831C3681BBADE
:10F01000C2F87C318378002C14BF4FF042624FF06D
:10F0200040620BB142F4801203781B0403F4702396
:10F030001343054A0120C2F8703110BD034901EAAB
:10F040008343DCE7002010BD004002400000FC1FAD
:10F050000B4B4FF00062C3F870214FF48022C3F8CD
:10F060007421084AC3F878216FF48471A2F16632E2
:10F070000A44C3F87C21044AC3F87021704700BFDA
:10F0800000400240785634120000080C10F0040FC3
:10F090000A4B10D04FF48042C3F8A020C2064CBFE8
:10F0A000074A084A9A6310F00800074B1ABF01226A
:10F0B0001A70187070474FF48072F3E700900440A4
:10F0C00000010A000001090030D4FF1F38B50446D2
:10F0D000F9F7FAFB0C49E517C1E90045D1E900450C
:10F0E0002B0243EA14632202C1E90023074A0023EA
:10F0F0001360074A1360074AD3645360D364BDE8C2
:10F100003840F9F7DDBB00BF70CDFF1F2CCDFF1FCE
:10F1100028CEFF1F009003400D490E4A4FF4804354
:10F1200030B5C1F8A0300C4B00240025C3E90045E0
:10F1300000231360094A1360094AD3645360D364FF
:10F14000084B1B7813B94FF480738B6330BD00BF3D
:10F150000090044028CEFF1F70CDFF1F2CCDFF1F55
:10F160000090034030D4FF1F10B9024B0901196011
:10F17000704700BF68CDFF1F08B9084686E7704793
:10F1800030B9044BD3E90023100A40EA036070470A
:10F190000020704770CDFF1F08B9084696E77047FA
:10F1A0002A4941F23C0210B58B58294C43F00073B8
:10F1B0008B50284B5A6D42F004025A651A6822F0AF
:10F1C00018021A605A6D22F001025A65D3F88420A1
:10F1D00042F0C002C3F8842000214FF6FF72D964C8
:10F1E00059609A60D3F8802042F00102C3F8802071
:10F1F000D3F8802042F02002C3F88020D3F880208A
:10F2000042F01002C3F880205A6D42F001025A65A4
:10F210001A6842F008021A604FF4E06323636363E4
:10F220000D4B0E4A186943091B0100F01F001360C3
:10F23000FFF72CFF0846FFF749FF4FF48043C4F85F
:10F24000A0305720BDE8104000F022B80070044004
:10F250000090044000900340C8CDFF1F68CDFF1F01
:10F26000FEE74FF0E023084AC3F8082D074A4CF2A6
:10F270002053D3814DF62813D381138823F0010343
:10F280001B041B0C13807047008000000020054009
:10F29000802800F01F014FF001030F4A04DD8B406E
:10F2A000C2F88C31D3607047402804DD8B40C2F82F
:10F2B000883193607047202804DD8B40C2F8843188
:10F2C00053607047404200F01F0058BF41428B40DE
:10F2D000C2F880311360704700E100E0802800F040
:10F2E0001F024FF001030D4903DD9340C1F88C303C
:10F2F0007047402803DD9340C1F8883070472028CC
:10F3000003DD9340C1F884307047404200F01F0095
:10F3100058BF42429340C1F88030704700E100E09E
:10F32000074B1A78D2B2012A02D1222903D15A708E
:10F3300001225A7070472129FAD10022F7E700BF55
:10F34000A4C8FF1F70B5154611B91B4B197070BDCD
:10F35000022903D1184B01221A7070BD04291AD159
:10F36000154B5B78012B25D19488402C28BF402475
:10F3700000235E1CDBB2A34207D300231A460221FE
:10F380001846BDE8704000F047BF2A68D05C00F026
:10F39000C3F83346EDE7032906D1074A5378012B1A
:10F3A00008D100239370E9E7052901BF024B002231
:10F3B0001A705A7070BD00BFA4C8FF1F10B5044674
:10F3C000204600F0C1F80028FAD110BD704738B5CA
:10F3D0000A4C012502460B4600202946A57000F084
:10F3E000F5FA224618B10023A370122038BD937895
:10F3F00003F0FF00002BFAD138BD00BFA4C8FF1FE7
:10F40000F8B506460F4600F0F4FC0E4B1A78012AB8
:10F4100016D15B78012B13D100F000F988B10025DB
:10F42000ECB2A74205D821463046BDE8F840FFF7C8
:10F43000CEBF301900F0D6F801350028F0D0F2E741
:10F440000C20F8BDA4C8FF1F08B540210248FFF7F3
:10F45000D7FF00F095F808BDA7C8FF1F38B50546CF
:10F4600000F0A8F80B28044609D140210548FFF711
:10F47000C7FF28B92846BDE8384000F09BB80024F3
:10F48000204638BDE7C8FF1F70B50C46461E002554
:10F490000CB9284670BD16F8010FFFF7DFFF013CDD
:10F4A000002818BF0B25A4B2F2E738B5451E00248A
:10F4B00015F8010F08B9204638BDFFF7CFFF002827
:10F4C00018BF0B24F4E707B5012300220093064977
:10F4D000064B104600F020FA002814BF1B20002025
:10F4E00003B05DF804FB00BF45F3000021F300000A
:10F4F00038B50C46054600F097F8A0420AD32C44D4
:10F500000020A54207D000B138BD15F8010B00F06E
:10F5100051F8F6E70B2038BD10B50A4A117840299A
:10F520000ED05378D4180133DBB2402BA07001F118
:10F5300001014FF00000117014BF5370507010BDE6
:10F540000B2010BD27C9FF1F10B50C4A117891B1CF
:10F5500092F84230D4180133DBB2A4780470402B07
:10F560004FF0000001F1FF31117014BF82F84230FA
:10F5700082F8420010BD0A2010BD00BF27C9FF1F3E
:10F58000014B1878704700BF27C9FF1F024B18783E
:10F59000C0F14000C0B2704727C9FF1F034B0022D3
:10F5A0005A7083F842201A70704700BF27C9FF1FA6
:10F5B000FFF7F4BF10B50A4A117840290ED05378EE
:10F5C000D4180133DBB2402BA07001F101014FF0E0
:10F5D0000000117014BF5370507010BD0B2010BD8F
:10F5E0006AC9FF1F10B50C4A117891B192F84230E8
:10F5F000D4180133DBB2A4780470402B4FF0000024
:10F6000001F1FF31117014BF82F8423082F84200DC
:10F6100010BD0A2010BD00BF6AC9FF1F014B18783A
:10F62000704700BF6AC9FF1F024B1878C0F1400045
:10F63000C0B270476AC9FF1F034B00225A7083F89B
:10F6400042201A70704700BF6AC9FF1FFFF7F4BF5E
:10F6500070B50546007801F093F902780023D9B21D
:10F66000914207D25C1C03EB830303445E786B7802
:10F670009E4227D1174C2B7A342202FB0142D678C6
:10F6800013B334234B43E218907886420CD000F039
:10F69000030204330C2010FB02302118205C0B897C
:10F6A0004A68497800F090FBD4F89C3083B12A4630
:10F6B000287812F8081F00290CBF03210521BDE896
:10F6C000704018472346CAE7937801339370D8E710
:10F6D00070BD00BFB0C9FF1F2DE9F04F85B00D46CA
:10F6E00090468DF80F0001F04BF9022D064647D1E8
:10F6F000077800235C1CDBB2BB4210DB4FF0000933
:10F70000DFF8B0B0CA465FFA89F4A74212DC284B92
:10F71000D3F89C30002B45D105B0BDE8F08F03EB4A
:10F72000830333440DF10F00DA78597801F0E2F9E0
:10F730002346DFE704EB84043444E378A28861784D
:10F74000CDF804A0A07800900DF10F0001F0B0F901
:10F75000A378032B05D15A4661789DF80F0001F07C
:10F7600031FA6178E37841F0100141EAC3110022D7
:10F77000C9B20DF10F0001F0EDF909F10109C2E77D
:10F78000002DC4D10A490378342000FB03138A1CDE
:10F790003633294634329A42B9D002F8341C02F882
:10F7A000331CF7E7424629469DF80F009847B3E718
:10F7B000B0C9FF1F51F60000F0B40C7804F06004EB
:10F7C000202C1D4632D14C78042C1DD00AD8012C97
:10F7D00004D003D3022C20D0032C12D00020288088
:10F7E000F0BC7047212C1BD004D8202CF6D1F0BCE3
:10F7F00000F040B9222C16D0232CEFD1F0BC00F041
:10F8000049B9F0BC00F049B902241C8014680025F5
:10F8100025701468671C17606570F0BC00F056B95D
:10F82000F0BC00F01FB9F0BC00F076B9402C06D156
:10F83000044CD4F8A04014B1A446F0BC6047CD20DD
:10F84000CEE700BFB0C9FF1F73B50446007801F0D2
:10F8500097F863680093A27A637A43EA0223ADF8CB
:10F86000043002780023D9B2914207D25D1C03EB29
:10F87000830303445E7863789E4225D1174D237A33
:10F88000342202FB0152D67803B334234B43EA18E7
:10F89000907886420CD000F0030204330C2010FB59
:10F8A00002302918285C0B894A68497800F08CFAE4
:10F8B000D5F89C3033B1227A20785AB104F108028D
:10F8C0000521984702B070BD2B46CCE793780133F1
:10F8D0009370DAE76A460321F3E700BFB0C9FF1F60
:10F8E00007B543680093437A817A43EA0123ADF870
:10F8F0000430084BD3F89C3002462BB1017A0078D3
:10F9000029B108320521984703B05DF804FB6A4627
:10F910000421F8E7B0C9FF1F2DE9F84305460F465B
:10F920001646984601F02CF802789DF820300132F6
:10F930008146D2B20021284601F09EF80446E8B97B
:10F94000164A1749284600F086F999F80000154B29
:10F95000342200FB022209F101011A449946343392
:10F96000934201F105010CD14146284600F074F89C
:10F97000044618B9C9F89C70C9F8A0602046BDE8D3
:10F98000F88311F8050C03F8340C11F8040C03F893
:10F99000330C03F8324C03F8314CE0E7B9F70000C0
:10F9A000D9F60000B0C9FF1F08B5074B0022C3F805
:10F9B0009C20C3F8A02000F0A1F918B9BDE80840C8
:10F9C00001F06EB808BD00BFB0C9FF1F2DE9F041BE
:10F9D000984605460E46174600F0D2FF04780023ED
:10F9E000D9B2A14207D2013303EB8302024412F8D9
:10F9F000042CB242F4D1174C34234B43E218D07894
:10FA000092F802E0A0EB0E01C9B2042902D1C12094
:10FA1000BDE8F08100F003010130C0B24FF00C0CE2
:10FA20000CFB0133D070A0EB0E001C44C0B20128C7
:10FA300025716671A760A4F80C8007D143463A4649
:10FA400031462846BDE8F04100F0BEB90020BDE8CF
:10FA5000F08100BFB0C9FF1F014B00201960704743
:10FA600054CAFF1F024B0979197100F08DBF00BF06
:10FA700054CAFF1F13B5002402AA1C80044B42F88D
:10FA8000041D0979197100F08DFF02B010BD00BF8F
:10FA900054CAFF1F00201880704730B40C46022162
:10FAA000198021796488084D012C297102D130BC5C
:10FAB00000F08EBF022C02D130BC00F095BF0020B8
:10FAC000188030BC704700BF54CAFF1F30B40C46CA
:10FAD0000221198021796488074D012C297102D1F6
:10FAE00030BC00F08DBF022C02D130BC00F09ABFB8
:10FAF0000020188030BC704754CAFF1F044B054AD1
:10FB000019795B791171137203210A23FFF75EBF24
:10FB100054CAFF1F4CC0FF1FF8B500271F808B7809
:10FB20000B4CA371C3F340035A0063F30002064673
:10FB30006271FFF7E3FF256845B1A37913F0020274
:10FB40001ABF3A46222121213046A8470020F8BD9D
:10FB500054CAFF1F034B00F108021B6800780521FF
:10FB6000184700BF5CCAFF1F70B5094D04462A1D27
:10FB7000012100F0D7FF80220121204600F0EAFF9A
:10FB80002B68207800220A21BDE87040184700BF8A
:10FB90005CCAFF1F37B501210DF10702044600F0D2
:10FBA000C1FF9DF80730074D802B04D12A79012130
:10FBB000204600F0CFFF2B68207800220B219847C9
:10FBC00003B030BD5CCAFF1F436805215A7800F0BE
:10FBD000C1BF73B50122002405460126002100F0B3
:10FBE00089FF334621468DE850001022284600F058
:10FBF0005FFF22462146284600F07CFF234621462F
:10FC00008DE850001022284600F052FF31460222B3
:10FC1000284600F09FFF32460621284600F09AFF52
:10FC200022469021284600F095FF044B28781B6857
:10FC30002246214602B0BDE8704018475CCAFF1F4B
:10FC400042783AB9C178C90141F0100101F0900140
:10FC500000F080BF704773B50C468DF8070001F0C7
:10FC60000DFA1F4D2C600446002836D11D4A9DF820
:10FC70000700102100F0A6FF1B4A044612219DF840
:10FC8000070000F09FFF194A044314219DF8070064
:10FC900000F098FFE4B20443154A9DF807001321D1
:10FCA00000F090FFE4B20443124A9DF807001721C8
:10FCB00000F088FF02AEE4B204430F4A16F8010DCB
:10FCC000162100F07FFFE4B20443032201213046F5
:10FCD00000F040FF0323E4B22B71204602B070BD58
:10FCE0005CCAFF1FD3FB0000C9FB000069FB0000DA
:10FCF00095FB000041FC000055FB000037B502AD4C
:10FD0000174B05F8010D0022102128461A6000F05B
:10FD10005BFF12210446284600F056FF14210443DD
:10FD2000284600F051FFE4B204431321284600F0B6
:10FD30004BFFE4B204431721284600F045FFE4B22C
:10FD400004431621284600F03FFFE4B2204310F0A0
:10FD5000FF0003D19DF8070001F09CF903B030BD0E
:10FD60005CCAFF1F1FB501218DF807000DF10E02BF
:10FD70000DF1070000F0D6FE0DF10F0206210DF186
:10FD8000070000F0CFFE9DF80E30802B18D19DF8B3
:10FD90000F309B0714D59DF8070000F0EFFD0128F8
:10FDA00004460DD172B60DF1070000F029FB0022C8
:10FDB00021460DF107008DF80E2000F0CBFE62B653
:10FDC0009DF80E0004B010BD73B50C4615461E46D6
:10FDD0008DF80700FFF7C6FF802808D033462A4673
:10FDE00021460DF1070000F0A7FA02B070BD002017
:10FDF000FBE77047062812D880000129C0B201D164
:10FE00000230C0B2074AC0F34703122101FB0323AB
:10FE10001A884FF6FF739A4208BFFF207047FF20F1
:10FE2000704700BF64CAFF1F2DE9F041314C324DCD
:10FE3000324E4FF0000884F800814FF4107285F8BC
:10FE400040020F462846FF2102F072F94FF480620B
:10FE500041463046C5F8446202F06AF994F80C3124
:10FE600043F0800384F80C3194F80C311B06FBD46A
:10FE7000234BFF221A7094F80C3143F0400384F8AE
:10FE80000C31204B196897B341F000411960194BB0
:10FE9000310AC6F3074201F0FE0183F89C1083F893
:10FEA000B020320E83F8B420174AC5F84822102239
:10FEB00083F80821012283F89420BF2283F8802050
:10FEC00093F8002102F07F0283F8002193F8842048
:10FED00042F0010283F8842093F8842042F010025B
:10FEE00083F8842084221A770020BDE8F08121F075
:10FEF0000041CBE70020074064CAFF1F00D6FF1F68
:10FF000056C0FF1F0070044000D8FF1F0D4B93F830
:10FF10000C2102F0BF0283F80C21BF2283F880205D
:10FF200093F8842002F0FE0283F8842093F8942052
:10FF300002F0FE0283F894201A7F02F07B021A7707
:10FF40000020704700200740F7B5082304248DE8FF
:10FF50001800B1F803300D788878B3F5007F81BFC1
:10FF60000023CB7002230B71062D71D8AB00DCB2DD
:10FF7000012804BF0234E4B24FEA540E354C122774
:10FF800007FB0E474FF6FF76B7F800C0B4455FD1C8
:10FF90004E78032E5CD801285AD897F80FC0BCF1D0
:10FFA000FF0F04BF4FF0000C87F80FC0B1F803C07B
:10FFB000122101FB0EFE04EB0E0743EA4003BA7365
:10FFC000FA7B7E7402F0010213435BB2D4F848223C
:10FFD000C7F80220D9B2F9733874D4F8447224F8FF
:10FFE0000EC01BB207EBC30E81F00101CEF8042056
:10FFF000AEF802C04FF0080E07F833E007EBC10E71
:020000021000EC
:10000000CEF80420AEF802C012FA8CF24FF0480E7F
:1000100007F831E0C4F8482228B917F8332062F015
:100020007F0207F8332002AA02EB80002DB20A49B2
:1000300050F8082C11F82530012E0CBF164642F05E
:1000400001063343DBB201F82530002003B0F0BDD8
:100050009520FBE764CAFF1FC0200740084610B583
:100060001146FFF7C7FEFF281DD0104B1221C0F329
:10007000470001FB0030D3F84422C37B1CB283F05D
:10008000010312F8341001F07F0102F8341012F865
:10009000331001F07F0102F833104FF0FF33837209
:1000A000C372002010BDC42010BD00BF64CAFF1F72
:1000B00073B50C468DF80700114620461646FFF72B
:1000C00099FEFF28054620D0214632460DF1070053
:1000D000FFF7C4FFC5F3470312210D4D59436B18B9
:1000E000D5F848221888121AC5F8482224B2094ABD
:1000F000002002F824004FF0FF326A549A705A70C0
:10010000DA701A715A7102B070BD9620FBE700BF19
:1001100064CAFF1FC02007402DE9F0410E4680460B
:10012000114630461746FFF765FE0C4DC0F34700F9
:10013000122303FB0050C47BFF2C0DD03A463146FE
:100140004046FFF78BFF24B2D5F8442212F8343032
:1001500063F07B0302F83430BDE8F08164CAFF1F0E
:1001600010B5084600211446FFF744FE084AC0F3C4
:100170004700122101FB0020D2F84432C27B03EB7E
:10018000C2035A68136823605368636010BD00BFE0
:1001900064CAFF1F10B50C4620461146FFF72AFE21
:1001A000FF281AD024B2104B13F82430DBB213F01E
:1001B0000C0F12D09B0712D40C4BD3F8443213F817
:1001C0003020D2090DD180F00100C0B213F83030D8
:1001D000DB0914BF0320002010BD052010BD012045
:1001E00010BD032010BD00BFC020074064CAFF1F20
:1001F00008B5FFF7FFFD074A1223C0F3470003FBD2
:100200000020C37BFF2B1EBFD2F84422002102F83E
:10021000331008BD64CAFF1F2DE9F04108460021D4
:1002200090461F46FFF7E6FD2249C0F3470012241F
:1002300004FB0014E57BFF2D39D022884FF6FF70B8
:1002400093B2834233D0D1F8441285F0010011F902
:10025000300000282BDB2EB287B901EBC6033846ED
:100260005A80D4F802205A6011F8352002F040027A
:1002700062F0770201F83620BDE8F08101EBC6029A
:10028000BB424FF0000028BF3B466781C4F80680A0
:10029000207360735380C2F8048011F8353003F086
:1002A000400363F0770301F83630BDE8F081942015
:1002B000BDE8F08164CAFF1F2DE9F0410C460646F7
:1002C000114620461546FFF795FD194BC0F3470030
:1002D000122202FB003090F80FE0BEF1FF0F24D095
:1002E00027B2144A6CB1407C012D0CBF1421182197
:1002F000012818BF41F0010112F82700014302F85C
:10030000271012F827106FF3410102F82710D3F8D5
:100310004432002203F83E203DB92B462A462146AE
:100320003046BDE8F041FFF777BFBDE8F08100BF80
:1003300064CAFF1FC02007402DE9F0410C4620464B
:10034000012117469846FFF755FDFF2836D01C4B74
:10035000C0F34700122202FB0030D3F8446290F849
:100360000FE016F93E30002B28DB23B2154A12F8B5
:10037000235015F0020521D10188C0F806701FFA3C
:1003800088F242818A42D8BF11460FFA8EF206EBFC
:10039000C2030573457359805F602CB9C82306F802
:1003A00032302046BDE8F08116F83E3003F04003BD
:1003B00063F0770306F832302C46F2E79324F0E737
:1003C00064CAFF1FC0200740034B044883F89810FD
:1003D0000122114600F0BEBB00200740A4CCFF1F45
:1003E000054B0648002283F89420802283F80C21D4
:1003F0000121FF2200F0AEBB00200740A4CCFF1F6C
:1004000038B51A4C94F8002102F07F0284F80021DC
:1004100094F80C2102F0DF0284F80C2194F880207B
:1004200042F0200284F8802094F8842002F0DF0259
:1004300084F8842094F8942002F0DF0284F8942059
:1004400094F8942042F0040284F8942044F6206545
:10045000013DADB200F0BCFE002DF9D194F894300E
:1004600003F0FB0384F8943038BD00BF0020074040
:100470002DE9F04FD84DD94C95F8807095F884301F
:1004800095F8906087B0FF221F4094F840328DF8B5
:1004900009208DF80C308DF80D20002301210DF17D
:1004A000090204F510708DF80E3004938DF81530A4
:1004B0008DF816308DF80F308DF8143000F032FBC7
:1004C00095F80C31D907F6B20FD59DF80930802B7D
:1004D0000BD195F8003103F07F0385F8003195F8D2
:1004E0000C3103F0DF0385F80C317A0711D5BA4BD4
:1004F000042093F8A41093F8A02083F8800006ABA2
:1005000042EA012223F80E2D03A91220049300F0E1
:100510006DFBFB074BD5B04DB0480123BF2685F8D6
:10052000803085F8886095F89430002743F0020306
:1005300085F894304FF4107285F89870FF2185F893
:10054000007101F0F5FD4FF480623946D4F84402A1
:1005500001F0EEFDD4F8443203F50073C4F84832DC
:100560009F4BFF221A7095F8943003F0FD0385F835
:10057000943095F80C3143F0400385F80C319F23FB
:1005800085F88C6085F8843095F8943003F0DF03AB
:1005900085F8943003A9102000F028FB95F89430DA
:1005A00003F0DF0385F8943007B0BDE8F08F3D0716
:1005B00040F19380884B082283F880203309C6F3EA
:1005C000C000062B8DF80D308DF80F0000F2F4807E
:1005D000C6F3800202EB830208B10232D2B2D4F831
:1005E000446206EBC201C2F34705D1F804E0498832
:1005F000ADF81510122101FB0541CDF810E091F87E
:100600000FC08CF0010C81F80FC016F8321082F088
:10061000010A5FFA8AFAC1F380110FFA8AF881F0B1
:100620000101890106EBC80906F83810002800F01E
:10063000D980DFF8ACB19BB99BF8002082B9FF22CA
:1006400019468BF8002003A81A460193FFF706FD10
:10065000019B06F838301A46194603A8FFF7DCFD5F
:100660009BF80030012B04D09DF80D30002B00F0DA
:10067000AD80122101FB0541BDF815008B894A8927
:1006800003449BB293428B8109D3B1F800E0C0B21E
:10069000864540F09380897B012940F08F801221AC
:1006A00001FB0544D4F8061020881944D31A83426C
:1006B000D8BF98B2A9F80200C9F8041016F83A3069
:1006C00003F0400363F0770306F83830424A92F8AB
:1006D000943003F0DF0382F89430B80717D53E4C0E
:1006E000022384F8803094F8883094F88C2003A991
:1006F000134016208DF8143000F078FABF2384F8E8
:10070000883094F8943003F0DF0384F89430F906CD
:100710001CD5314C202384F88030102384F880309D
:1007200003A9142000F062FA94F80C3143F020037E
:1007300084F80C3194F8003143F0800384F80031E0
:1007400094F8843043F0200384F88430BA060DD541
:10075000214C202384F8803003A9132000F046FAAE
:1007600094F8843003F0DF0384F884303B067FF58F
:100770001BAF0DF10A02FF23102103A88DF80D30E5
:1007800000F0D0F99DF80A30134C012B04BF8DF80E
:100790000F3000224FF0800308BF8DF80D2003A911
:1007A00084F88030172000F021FA94F8943003F098
:1007B000DF0384F89430F7E6FF2210E7122202FBF1
:1007C0000544D4F806200492ADF8153003A99DF82D
:1007D0000D0000F00BFA79E70020074064CAFF1F04
:1007E00056C0FF1F6BB916F832202F4902F03C02A9
:1007F000342A35D101238DF80E309EF80030DB0904
:100800000B70122101FB05414FF6FF734A899A4292
:10081000DCD0BDF815E08B8973449BB28B810988CD
:100820008E4501D19A420CD88AB3B2FBF1F001FB9C
:10083000102080B258BB122000FB0540807B0128AD
:1008400025D1D21A8A42D8BF91B2122202FB0544A6
:10085000C9B9D4F80230C9F80430A9F802102DE75C
:100860000A78012ACDD1FF200870194603A8019308
:10087000FFF7F4FB019B06F838301A46194603A827
:10088000FFF7CAFCBDE7D4F806201344E3E71222C1
:1008900002FB0544D4F80620ADF815304FF0FF33C5
:1008A0000492A372E37291E756C0FF1F13460A46F3
:1008B000194601F03DBC00BF30B50329039C0498E4
:1008C0001DD12BB9164A226004220280002030BDBF
:1008D00040F209418B420FD1022A4FF000030CD89D
:1008E00010490C2505FB0313D9681B6951F8221028
:1008F00021609B5C0380E9E701230122F0E70729DF
:1009000001D9CD2030BD074B03EB8102126A226072
:10091000002AF6D003EB4103B3F84030EAE700BF0A
:1009200057C0FF1F6C23010001299FBF034B5B5C75
:100930001370002088BFCD20704700BFB0CCFF1FD0
:1009400001299DBF024B00205A54CD20704700BFA3
:10095000B0CCFF1F19B14B1E5842584170470120BF
:100960007047054B1A788A4204D05878431A584287
:100970005841704701207047B0CCFF1F00207047DE
:1009800000487047BC23010001299FBF044BC1EB05
:10099000C101C918002094BF1160CD20704700BF6D
:1009A0005BC0FF1F012930B50ED8084DC1EBC10156
:1009B00008231068C45CC818284401330F2B00F8C2
:1009C000084CF6D1002030BDCD2030BD5BC0FF1FEC
:1009D00001299FBF034B03EB41010020116088BF39
:1009E000CD207047B2CCFF1F01299FBF034B03EB03
:1009F00041010020116088BFCD207047B6CCFF1F99
:100A000001290AD813681878054B03EB4101887057
:100A100013685B78CB7000207047CD20704700BF13
:100A2000B0CCFF1F01290AD813681878054B03EBD7
:100A30004101887113685B78CB7100207047CD202D
:100A4000704700BFB0CCFF1F084B5A7803F8022B49
:100A5000FF210022D1540132072AFBD1044A00238E
:100A6000052199540133072BFBD17047BACCFF1FE6
:100A7000C3CCFF1F00BF7047013AD2B2062A10B59F
:100A80001C4608D8054B5A70FFF7DEFF2146BDE82B
:100A90001040FFF7C9B9992010BD00BFBACCFF1FA5
:100AA000024B00225A70FFF731BA00BFBACCFF1FC9
:100AB00037B50F4C257805B9C1B98DF802308DF8DE
:100AC00000109DF81830ADF8032069469DF81C20F1
:100AD00000788DF80130FFF737FA9DF800301BB130
:100AE00010B92378013B237003B030BD9520FBE79C
:100AF000BACCFF1F38B50A4B0D461C7859788C428A
:100B00001C4600D14DB929460078FFF7D1FA2DB126
:100B100020B923780133237038BD962038BD00BF3B
:100B2000BACCFF1F4B1E062B05D8094B19444B7836
:100B3000137000207047CB0607D501F00F0106297E
:100B400003D8034B19444B7AF2E78220704700BF69
:100B5000BACCFF1F4B1E062B2DE9F04180461746ED
:100B600005D8174B19444A700020BDE8F081CB0628
:100B700022D501F00F05062D1ED8012A4FEAD11407
:100B80000F4E06D122462946FFF7C6FA35446F724A
:100B9000EAE7002AFAD173195B7A012BF6D12246D3
:100BA0002946FFF789FB002DF0D184F00102294688
:100BB0004046FFF781FBE9E78220BDE8F08100BFF6
:100BC000BACCFF1F00207047062903D9A1F11003FA
:100BD000072B07D8044B53F82130002B0CBFC4203F
:100BE00000207047C4207047E4230100102810B58E
:100BF0000C4601D1FFF728FF034B53F820300BB10F
:100C000020469847002010BDE42301001FB514467C
:100C100002228DF807001A8005210DF10F020DF157
:100C20000700FFF77FFF034B9DF80F201A8023601A
:100C300004B010BDCCCCFF1F1FB5144601228DF8A7
:100C400007001A8004210DF10F020DF10700FFF7D4
:100C500069FF044B9DF80F201A800020236004B028
:100C600010BD00BFCCCCFF1FF0B5002685B01E80A4
:100C700049888DF80700ADF80E10FFF76BFE18B32A
:100C8000BDF80E20114F04ACB2FA82F252090121D4
:100C90000DF10700FFF75EFF34F8022D0421D2B2F8
:100CA0000DF10700FFF756FF7B682246012105463C
:100CB0009DF8070098477B689DF80700324602219F
:100CC0009847284605B0F0BD0425FAE7CCCCFF1FB5
:100CD00073B502AC002504F8010D0E461D800422F8
:100CE00001212046FFF736FF7288024B28461A7210
:100CF00002B070BDCCCCFF1F13B54C8889888DE83D
:100D00000C000B46E2B2210AFFF7D6FD02B010BD7F
:100D10002DE9F04186B017461E4606AA00238846F4
:100D2000059303238DF80F0002F8083D01210DF112
:100D30000F00FFF7F7FE98F80050274C15F0030559
:100D400028D10DF1110206210DF10F00FFF7EAFE87
:100D50009DF811309DF80F0003F0030323800DF17F
:100D60001203019305AB00932A462B460221FFF79D
:100D7000A3FD059BDB7913F0400F238814BF43F0DC
:100D8000010323F001032380022333803C6006B07B
:100D9000BDE8F081012D08D19DF81030012B02D162
:100DA00098F80430ABB90023EDE7022DEED198F8A6
:100DB000041041F010010DF11202C9B20DF10F0043
:100DC000FFF7B0FE9DF8123003F001032380358059
:100DD000DCE7CD20DAE700BFCCCCFF1F7FB50022D7
:100DE0001A800B784E788DF8070013F003030D4638
:100DF000C6F3400634D1FEB14B88013B9BB2012BB8
:100E000052D80DF10F0206210DF10700FFF78AFEFF
:100E1000044670B9AB7801229A409DF80F301A430E
:100E2000D2B206210DF107008DF80F20FFF792FED8
:100E30000446204604B070BD4E88012E34D10DF119
:100E40000F0206210DF10700FFF76CFE0446002893
:100E5000EFD1AA7896409DF80F2022EA0602E0E73B
:100E6000022B21D109798DF80F10324641F0100183
:100E70000DF10700FFF76EFE6B78002E14BF0721FF
:100E80000821012B044607D19DF80F00C10900F08D
:100E90000F00FFF7ADF90821044B9DF807005B68D0
:100EA0000DF10F029847C4E7CD24C2E7CCCCFF1F59
:100EB00010B500241C800B7803F00303012B05D12F
:100EC0008A780979FFF73CFD204610BD042010BD4B
:100ED00038B515460A7802F00302012A07D1054CFD
:100EE0001A8009792246FFF71FFD2C6038BD0420C7
:100EF00038BD00BFCCCCFF1F13B5CD298DF807003E
:100F000007D1012290210DF10700FFF723FE02B067
:100F100010BD0D491C88088A1268844288BF188059
:100F20000C461B889DF807000021FEF74DFF94F941
:100F30000A30002BEBDA00231A4619460DF10700A0
:100F4000FFF76AF9E3E700BFCCCCFF1F73B5054696
:100F500000266A4601218DF800600196FFF7E2FD48
:100F6000AA78434C012A52D168680368C4F80A3051
:100F70004368A07AC4F80E3004F10A0110F0600F43
:100F80001ED1E27A3B4B53F82240002C3DD09DF815
:100F90000000022839D802EB42021344034493F8BC
:100FA0003430012B31D10DF1020301AA2878A0477A
:100FB0000DF1020301AA01462878FFF79DFF13E017
:100FC000238AADF80230202B17D87BB102060DD44E
:100FD0000A68C4F812204A68C4F81620314604F1A1
:100FE0001A022846FFF718F902B070BDE46B64B12D
:100FF0000DF1020301AA2049D8E702A82B7800F8D6
:10100000073D9021FFF7A6FDEEE7CD20D0E79DF844
:101010000030042B10D12B78217A02AD05F8063D63
:101020002846FFF7D1F9012211462846FFF792FD25
:10103000227A03212846E5E794F90A30002BD3DB16
:10104000EB78002BD0D1E66B86B1B5F80930287863
:101050000833ADF8023004F112010DF1020301AAC8
:10106000B04701460DF1020301AAA5E7CD21F9E73A
:10107000CCCCFF1F44240100D6CCFF1F034B59608A
:10108000DA630021024AFFF79DBD00BFCCCCFF1FF1
:101090004D0F010007B502AB054A03F8010D002111
:1010A00018465160D163FFF78FFD03B05DF804FB74
:1010B000CCCCFF1F00207047354B41F248015A58F5
:1010C00022F00D0242F005025A5041F204015A5832
:1010D00042F480225A5041F234015A5842F480229C
:1010E0005A5003F52C33602193F8942042F0020209
:1010F00083F89420C02283F80021FF221A7483F819
:10110000802083F8882083F88420002283F88C20B4
:1011100083F80C111F491A75080A00F0FE0083F8C5
:10112000982083F8C02083F8C42083F8C82083F86F
:10113000CC2083F8D02083F8D42083F8D82083F8FB
:10114000DC2083F8E02083F8E42083F8E82083F8AB
:10115000EC2083F8F02083F8F42083F8F82083F85B
:10116000FC2083F89C00C1F30740090E83F8B0000F
:1011700083F8B41083F8AC201A7783F8082193F829
:10118000942002F0D40242F0010283F894207047C8
:101190000070044000D6FF1F024B4FF400729A60AB
:1011A000704700BF00E100E0034B4FF40072C3F84A
:1011B00088219A60704700BF00E100E008B5FEF7A3
:1011C00082F910B9FFF7F0FF08BD1B2008BD00BF72
:1011D000034B4AF202629A814BF280429A81704735
:1011E0000020054081F0004102E000BF83F0004391
:1011F00030B54FEA41044FEA430594EA050F08BFB2
:1012000090EA020F1FBF54EA000C55EA020C7FEA75
:10121000645C7FEA655C00F0E2804FEA5454D4EBF2
:101220005555B8BF6D420CDD2C4480EA020281EABC
:10123000030382EA000083EA010180EA020281EAF4
:101240000303362D88BF30BD11F0004F4FEA013146
:101250004FF4801C4CEA113102D0404261EB410155
:1012600013F0004F4FEA03334CEA133302D05242DB
:1012700063EB430394EA050F00F0A780A4F1010497
:10128000D5F1200E0DDB02FA0EFC22FA05F28018D1
:1012900041F1000103FA0EF2801843FA05F35941B7
:1012A0000EE0A5F120050EF1200E012A03FA0EFC36
:1012B00028BF4CF0020C43FA05F3C01851EBE37160
:1012C00001F0004507D54FF0000EDCF1000C7EEB7D
:1012D00000006EEB0101B1F5801F1BD3B1F5001FBB
:1012E0000CD349085FEA30004FEA3C0C04F10104DA
:1012F0004FEA445212F5800F80F09A80BCF1004F03
:1013000008BF5FEA500C50F1000041EB045141EA84
:10131000050130BD5FEA4C0C404141EB010111F485
:10132000801FA4F10104E9D191F0000F04BF014630
:101330000020B1FA81F308BF2033A3F10B03B3F10E
:1013400020020CDA0C3208DD02F1140CC2F10C029E
:1013500001FA0CF021FA02F10CE002F11402D8BFFC
:10136000C2F1200C01FA02F120FA0CFCDCBF41EAC8
:101370000C019040E41AA2BF01EB0451294330BD97
:101380006FEA04041F3C1CDA0C340EDC04F1140474
:10139000C4F1200220FA04F001FA02F340EA03004B
:1013A00021FA04F345EA030130BDC4F10C04C4F191
:1013B000200220FA02F001FA04F340EA0300294671
:1013C00030BD21FA04F0294630BD94F0000F83F4BB
:1013D000801306BF81F480110134013D4EE77FEA9E
:1013E000645C18BF7FEA655C29D094EA050F08BFEA
:1013F00090EA020F05D054EA000C04BF19461046CB
:1014000030BD91EA030F1EBF0021002030BD5FEA0E
:10141000545C05D14000494128BF41F0004130BD36
:1014200014F580043CBF01F5801130BD01F000458A
:1014300045F0FE4141F470014FF0000030BD7FEAFD
:10144000645C1ABF194610467FEA655C1CBF0B46F8
:10145000024650EA013406BF52EA033591EA030F0F
:1014600041F4002130BD00BF90F0000F04BF002107
:10147000704730B54FF4806404F132044FF000053A
:101480004FF0000150E700BF90F0000F04BF0021B3
:10149000704730B54FF4806404F1320410F0004519
:1014A00048BF40424FF000013EE700BF42004FEA14
:1014B000E2014FEA31014FEA02701FBF12F07F4391
:1014C00093F07F4F81F06051704792F0000F14BF8E
:1014D00093F07F4F704730B54FF4607401F00045D2
:1014E00021F0004120E700BF50EA010208BF704729
:1014F00030B54FF000050AE050EA010208BF70471E
:1015000030B511F0004502D5404261EB41014FF486
:10151000806404F132045FEA915C3FF4DCAE4FF08A
:1015200003025FEADC0C18BF03325FEADC0C18BF71
:10153000033202EBDC02C2F1200300FA03FC20FAC2
:1015400002F001FA03FE40EA0E0021FA02F114440F
:10155000C1E600BF70B54FF0FF0C4CF4E06C1CEA24
:1015600011541DBF1CEA135594EA0C0F95EA0C0F99
:1015700000F0DEF82C4481EA030621EA4C5123EA0C
:101580004C5350EA013518BF52EA033541F480113B
:1015900043F4801338D0A0FB02CE4FF00005E1FBEE
:1015A00002E506F00042E0FB03E54FF00006E1FB38
:1015B00003569CF0000F18BF4EF0010EA4F1FF047B
:1015C000B6F5007F64F5407404D25FEA4E0E6D41BB
:1015D00046EB060642EAC62141EA55514FEAC520CC
:1015E00040EA5E504FEACE2EB4F1FD0C88BFBCF548
:1015F000E06F1ED8BEF1004F08BF5FEA500E50F1F9
:10160000000041EB045170BD06F0004646EA0101BE
:1016100040EA020081EA0301B4EB5C04C2BFD4EBF0
:101620000C0541EA045170BD41F480114FF0000EE9
:10163000013C00F3AB8014F1360FDEBF002001F057
:10164000004170BDC4F10004203C35DA0C341BDCD1
:1016500004F11404C4F1200500FA05F320FA04F0A3
:1016600001FA05F240EA020001F0004221F00041D7
:1016700010EBD37021FA04F642EB06015EEA430E4A
:1016800008BF20EAD37070BDC4F10C04C4F120057A
:1016900000FA04F320FA05F001FA04F240EA02002D
:1016A00001F0004110EBD37041F100015EEA430EFE
:1016B00008BF20EAD37070BDC4F1200500FA05F21E
:1016C0004EEA020E20FA04F301FA05F243EA02039D
:1016D00021FA04F001F0004121FA04F220EA0200AC
:1016E00000EBD3705EEA430E08BF20EAD37070BDF2
:1016F00094F0000F0FD101F00046400041EB0101D2
:1017000011F4801F08BF013CF7D041EA060195F0B3
:10171000000F18BF704703F00046520043EB03036D
:1017200013F4801F08BF013DF7D043EA060370475A
:1017300094EA0C0F0CEA135518BF95EA0C0F0CD065
:1017400050EA410618BF52EA4306D1D181EA0301AB
:1017500001F000414FF0000070BD50EA410606BFA5
:101760001046194652EA430619D094EA0C0F02D1EA
:1017700050EA013613D195EA0C0F05D152EA03362F
:101780001CBF104619460AD181EA030101F000414D
:1017900041F0FE4141F470014FF0000070BD41F096
:1017A000FE4141F4780170BD70B54FF0FF0C4CF470
:1017B000E06C1CEA11541DBF1CEA135594EA0C0F8F
:1017C00095EA0C0F00F0A7F8A4EB050481EA030EDC
:1017D00052EA03354FEA013100F088804FEA0333C3
:1017E0004FF0805545EA131343EA12634FEA022291
:1017F00045EA111545EA10654FEA00260EF0004152
:101800009D4208BF964244F1FD0404F5407402D2A3
:101810005B084FEA3202B61A65EB03055B084FEA34
:1018200032024FF480104FF4002CB6EB020E75EB31
:10183000030E22BFB61A754640EA0C005B084FEA59
:101840003202B6EB020E75EB030E22BFB61A7546D6
:1018500040EA5C005B084FEA3202B6EB020E75EB21
:10186000030E22BFB61A754640EA9C005B084FEA99
:101870003202B6EB020E75EB030E22BFB61A7546A6
:1018800040EADC0055EA060E18D04FEA051545EA95
:1018900016754FEA06164FEAC30343EA52734FEA3E
:1018A000C2025FEA1C1CC0D111F4801F0BD141EAB7
:1018B00000014FF000004FF0004CB6E711F4801F1C
:1018C00004BF01430020B4F1FD0C88BFBCF5E06FFC
:1018D0003FF6AFAEB5EB030C04BFB6EB020C5FEA0C
:1018E000500C50F1000041EB045170BD0EF0004E61
:1018F0004EEA113114EB5C04C2BFD4EB0C0541EA93
:10190000045170BD41F480114FF0000E013C90E68F
:1019100045EA060E8DE60CEA135594EA0C0F08BF53
:1019200095EA0C0F3FF43BAF94EA0C0F0AD150EA52
:1019300001347FF434AF95EA0C0F7FF425AF1046E5
:1019400019462CE795EA0C0F06D152EA03353FF40D
:10195000FDAE1046194622E750EA410618BF52EA8A
:1019600043067FF4C5AE50EA41047FF40DAF52EA5E
:1019700043057FF4EBAE12E74FEA410212F5001285
:1019800015D211D56FF47873B3EB625212D94FEAC6
:10199000C12343F0004343EA505311F0004F23FAB0
:1019A00002F018BF404270474FF00000704750EA05
:1019B000013005D111F0004008BF6FF000407047C2
:1019C0004FF00000704700BF4FEA4102B2F1E04320
:1019D00024BFB3F5001CDCF1FE5C0DD901F0004C16
:1019E0004FEAC0024CEA5070B2F1004F40EB830066
:1019F00008BF20F00100704711F0804F21D113F192
:101A00003872BCBF01F00040704741F480114FEACA
:101A10005252C2F11802C2F1200C10FA0CF320FA53
:101A200002F018BF40F001004FEAC1234FEAD32370
:101A300003FA0CFC40EA0C0023FA02F34FEA4303DA
:101A4000CCE77FEA625307D150EA01331EBF4FF063
:101A5000FE4040F44000704701F0004040F0FE407E
:101A600040F40000704700BF80F0004002E000BF7B
:101A700081F0004142001FBF5FEA410392EA030F79
:101A80007FEA226C7FEA236C6AD04FEA1262D2EBC3
:101A90001363C1BFD218414048404140B8BF5B42C8
:101AA000192B88BF704710F0004F40F4000020F061
:101AB0007F4018BF404211F0004F41F4000121F077
:101AC0007F4118BF494292EA030F3FD0A2F10102C1
:101AD00041FA03FC10EB0C00C3F1200301FA03F1FF
:101AE00000F0004302D5494260EB4000B0F5000F22
:101AF00013D3B0F1807F06D340084FEA310102F1E1
:101B00000102FE2A51D2B1F1004F40EBC25008BF92
:101B100020F0010040EA03007047490040EB00005C
:101B200010F4000FA2F10102EDD1B0FA80FCACF18B
:101B3000080CB2EB0C0200FA0CF0AABF00EBC2508A
:101B400052421843BCBFD0401843704792F0000F78
:101B500081F4000106BF80F400000132013BB5E7CB
:101B60004FEA41037FEA226C18BF7FEA236C21D041
:101B700092EA030F04D092F0000F08BF08467047A6
:101B800090EA010F1CBF0020704712F07F4F04D174
:101B9000400028BF40F00040704712F100723CBF87
:101BA00000F50000704700F0004343F0FE4040F4B1
:101BB000000070477FEA226216BF08467FEA23636F
:101BC0000146420206BF5FEA412390EA010F40F45A
:101BD000800070474FF0000304E000BF10F00043A6
:101BE00048BF40425FEA000C08BF704743F096438D
:101BF00001464FF000001CE050EA010208BF7047A8
:101C00004FF000030AE000BF50EA010208BF70472E
:101C100011F0004302D5404261EB41015FEA010C43
:101C200002BF84460146002043F0B64308BFA3F13B
:101C30008053A3F50003BCFA8CF2083AA3EBC2531D
:101C400010DB01FA02FC634400FA02FCC2F120023C
:101C5000BCF1004F20FA02F243EB020008BF20F073
:101C60000100704702F1200201FA02FCC2F12002D9
:101C700050EA4C0021FA02F243EB020008BF20EACE
:101C8000DC7070474FF0FF0C1CEAD0521EBF1CEAFC
:101C9000D15392EA0C0F93EA0C0F6FD01A4480EAEA
:101CA000010C400218BF5FEA41211ED04FF00063D3
:101CB00043EA501043EA5111A0FB01310CF00040FF
:101CC000B1F5000F3EBF490041EAD3715B0040EA25
:101CD000010062F17F02FD2A1DD8B3F1004F40EBF5
:101CE000C25008BF20F00100704790F0000F0CF0C8
:101CF000004C08BF49024CEA502040EA51207F3A8C
:101D0000C2BFD2F1FF0340EAC250704740F4000066
:101D10004FF00003013A5DDC12F1190FDCBF00F057
:101D200000407047C2F10002410021FA02F1C2F105
:101D3000200200FA02FC5FEA310040F1000053EAA1
:101D40004C0308BF20EADC70704792F0000F00F0EF
:101D5000004C02BF400010F4000F013AF9D040EAF5
:101D60000C0093F0000F01F0004C02BF490011F489
:101D7000000F013BF9D041EA0C018FE70CEAD15387
:101D800092EA0C0F18BF93EA0C0F0AD030F0004C07
:101D900018BF31F0004CD8D180EA010000F00040BB
:101DA000704790F0000F17BF90F0004F084691F079
:101DB000000F91F0004F14D092EA0C0F01D14202B3
:101DC0000FD193EA0C0F03D14B0218BF084608D17C
:101DD00080EA010000F0004040F0FE4040F40000C6
:101DE000704740F0FE4040F4400070474FF0FF0C59
:101DF0001CEAD0521EBF1CEAD15392EA0C0F93EAA0
:101E00000C0F69D0A2EB030280EA010C49024FEAF1
:101E1000402037D04FF0805343EA111143EA1013AA
:101E20000CF000408B4238BF5B0042F17D024FF462
:101E3000000C8B4224BF5B1A40EA0C00B3EB510F3D
:101E400024BFA3EB510340EA5C00B3EB910F24BF26
:101E5000A3EB910340EA9C00B3EBD10F24BFA3EBAB
:101E6000D10340EADC001B0118BF5FEA1C1CE0D173
:101E7000FD2A3FF650AF8B4240EBC25008BF20F026
:101E8000010070470CF0004C4CEA50207F32C2BF7A
:101E9000D2F1FF0340EAC250704740F400004FF017
:101EA0000003013A37E792F0000F00F0004C02BF48
:101EB000400010F4000F013AF9D040EA0C0093F012
:101EC000000F01F0004C02BF490011F4000F013B6C
:101ED000F9D041EA0C0195E70CEAD15392EA0C0FD4
:101EE00008D142027FF47DAF93EA0C0F7FF470AF0C
:101EF000084676E793EA0C0F04D14B023FF44CAF4F
:101F000008466EE730F0004C18BF31F0004CCAD1E3
:101F100030F000427FF45CAF31F000437FF43CAF1F
:101F20005FE700BF4FF0FF3C06E000BF4FF0010C41
:101F300002E000BF4FF0010C4DF804CD4FEA400223
:101F40004FEA41037FEA226C18BF7FEA236C11D06D
:101F500001B052EA530C18BF90EA010F58BFB2EB20
:101F6000030088BFC81738BF6FEAE17018BF40F0A0
:101F7000010070477FEA226C02D15FEA402C05D154
:101F80007FEA236CE4D15FEA412CE1D05DF8040BD9
:101F9000704700BF844608466146FFE70FB5FFF76C
:101FA000C9FF002848BF10F1000F0FBD4DF808ED24
:101FB000FFF7F4FF0CBF012000205DF808FB00BF15
:101FC0004DF808EDFFF7EAFF34BF012000205DF86F
:101FD00008FB00BF4DF808EDFFF7E0FF94BF0120BC
:101FE00000205DF808FB00BF4DF808EDFFF7D2FFB9
:101FF00094BF012000205DF808FB00BF4DF808EDFC
:10200000FFF7C8FF34BF012000205DF808FB00BFC8
:1020100042000ED2B2F1FE4F0BD34FF09E03B3EB52
:10202000126209D44FEA002343F0004323FA02F07E
:1020300070474FF00000704712F1610F01D142026A
:1020400002D14FF0FF3070474FF00000704700BFE3
:10205000FDF707F9002103E00A4B5B5843500431B8
:1020600009480A4B42189A42F6D3094A02E0002373
:1020700013600432074B9A42F9D300F00DF8804701
:1020800070470000D024010008C0FF1F6CC5FF1F6F
:1020900000C6FF1F24DAFF1F224C08B5F6F7F1F93E
:1020A000F6F758FAF6F70CFCF6F723FCF6F71EFBEA
:1020B000F6F7E6FEFCF754FEF7F765F9F6F7BCFC19
:1020C000E08CF6F7BAFD2078F6F72AFBE078F6F711
:1020D00097FBF6F7B1FE21896079228AFCF794FE1E
:1020E000F7F7A2FDF7F786FFFDF75AF80E4B04222B
:1020F0009A60FBF7C1F8FBF757FD0C4B20229A6062
:10210000FBF7B6F9FBF780FDFBF74FFDF6F748FE4E
:10211000F6F782FE0028F3D0F7F76CFFFBF7ACF878
:10212000EEE700BF0CC0FF1FC0F00F4000F10F40F2
:1021300070B4860746D0541E002A41D0CAB2034666
:1021400002E014F1FF343BD303F8012B9D07F8D1D3
:10215000032C2ED9CDB245EA05250F2C45EA0545BD
:1021600019D903F110022646103E0F2E42F8105CDA
:1021700042F80C5C42F8085C42F8045C02F1100280
:10218000F2D8A4F1100222F00F0204F00F04103272
:10219000032C13440DD91E462246043A032A46F85E
:1021A000045BFAD8221F22F003020432134404F025
:1021B00003042CB1C9B21C4403F8011B9C42FBD19F
:1021C00070BC704714460346C2E700BF024B13B110
:1021D000024800F005B8704700000000ED21010042
:1021E000002301461A46184600F01EB838B50A4CBE
:1021F0000A4D641BA4100AD004F18043013B05EB97
:102200008305013C55F804399847002CF9D1BDE805
:10221000384000F051B900BFD0240100CC240100A7
:10222000704700BF704700BF2DE9F8432C4D0646AC
:10223000286898460F469146FFF7F2FF294B1C6825
:10224000D4F84831002B3ED05A681F2A1CDC02F11A
:10225000010E76B103EB82010124C1F88890D3F816
:10226000880194402043022EC3F88801C1F80881F8
:1022700023D00232C3F804E0286843F82270FFF745
:10228000D1FF0020BDE8F883174B0BB34FF4C870A3
:10229000AFF300800346D8B1D4F848210260002192
:1022A00041600A46C4F848014FF0010EC0F8881199
:1022B000C0F88C11002EDCD0CCE7D3F88C110C4385
:1022C000C3F88C41D5E704F5A673C4F84831BBE7E1
:1022D0002868FFF7A7FF4FF0FF30BDE8F88300BF85
:1022E00068C5FF1FA8240100000000008025000031
:1022F00040380000004B0000807000000096000095
:1023000000E10000002C010000C201000084030075
:1023100090D0030020A1070040420F00F40100000C
:102320006400000001800808000000000064000054
:102330000000000000000000C800000000000000D5
:1023400000000000010003E800000000000000039E
:10235000E800000000000200FA0600030000000090
:1023600000370600000000000000000057C0FF1FFB
:102370000400000009040000D0230100E023010054
:10238000000000000000000000000000000000004D
:102390002EC1FF1FEBC0FF1F000000000000000067
:1023A000000000000000000000000000000012001B
:1023B00043000000000000000000000003010201D3
:1023C00010000202001000030301100000010000D1
:1023D00057C0FF1FB1C0FF1F8BC0FF1F69C0FF1F89
:1023E000043A26224D0F010049F80000E1F80000F0
:1023F00051F60000750A0100750A0100750A010016
:10240000750A0100750A0100750A0100750A0100CC
:10241000750A0100750A0100750A0100750A0100BC
:10242000750A0100D3FB000069FB0000C9FB000036
:1024300095FB000069FB0000750A010055FB0000D8
:1024400041FC0000110D0100DD0D01000000000045
:10245000DD0D010000000000D10C0100F90C0100AD
:1024600000000000390C0100690C0100D10E0100D0
:10247000B10E01000D0C010001010001010000007E
:102480000001010000000000010101010100000045
:102490000101000101000100000100000100003104
:1024A000313130563130390040C1FF1FF8B500BF1F
:1024B000F8BC08BC9E467047F8B500BFF8BC08BC25
:0424C0009E4670477D
:0824C400CD2101003584000068
:0424CC001184000077
:1024D0009F2401000001020000080000010000002C
:1024E00002000000000000000000000000000000EA
:1024F00000000000000000000000070000000000D5
:1025000000000000000000000000000000000000CB
:1025100000000000A1200000000002000000FF04F5
:1025200003090400C20100000008000000000000D0
:102530000022034200410044002000530054005296
:102540000049004E004700200049004E004400456D
:102550000058002603530074006500700070006589
:1025600000720020004D006F0074006F00720020A8
:102570000044006500760020003A035400520049F0
:10258000004E0041004D004900430020004D006F07
:1025900000740069006F006E00200043006F006E41
:1025A00000740072006F006C0020002000200020EA
:1025B00000200009024300020100C03209040000AB
:1025C000010202000005240010010524010101049C
:1025D00024020605240600010705830310000A09EA
:1025E000040100020A000000070581021000000734
:1025F00005020210000012010002020000103C2A35
:102600000001020001020001000000002CC4FF1FB5
:1026100094C4FF1FFCC4FF1F000000000000000066
:1026200000000000000000000000000000000000AA
:10263000000000000000000000000000000000009A
:10264000000000000000000000000000000000008A
:10265000000000000000000000000000000000007A
:10266000000000000000000000000000000000006A
:10267000000000000000000000000000000000005A
:10268000000000000000000000000000000000004A
:10269000000000000000000000000000000000003A
:1026A000000000000000000000000000000000002A
:1026B00001000000000000000E33CDAB34126DE6C7
:1026C000ECDE05000B000000000000000000000030
:1026D00000000000000000000000000000000000FA
:1026E00000000000000000000000000000000000EA
:1026F00000000000000000000000000000000000DA
:1027000000000000000000000000000000000000C9
:042A300000DAFF1FAA
:102A3400D024010008C0FF1F64050000000000004E
:082A440000000000000000008A
:020000020000FC
:020000041FFFDC
:04C00000000000003C
:040000031000205178
:00000001FF
